LX51 LINKER/LOCATER V4.66.97.0                                                          03/02/2021  17:27:53  PAGE 1


LX51 LINKER/LOCATER V4.66.97.0, INVOKED BY:
D:\KEILC51\C51\BIN\LX51.EXE .\Out_Files\STARTUP.obj, .\Out_Files\system_um800x.obj, .\Out_Files\common.obj, .\Out_Files\
>> uart0.obj, .\Out_Files\adc.obj, .\Out_Files\app.obj, .\Out_Files\main.obj TO .\Out_Files\adc PRINT (.\Out_Files\adc.m
>> ap) REMOVEUNUSED CLASSES (XDATA (X:0X0-X:0X7FF), HDATA (X:0X0-X:0X7FF), CODE (C:0X0-C:0X7FFF), CONST (C:0X0-C:0X7FFF)
>> , ECODE (C:0X0-C:0X7FFF), HCONST (C:0X0-C:0X7FFF))


CPU MODE:     8051 MODE
MEMORY MODEL: COMPACT WITH FLOATING POINT ARITHMETIC


INPUT MODULES INCLUDED:
  .\Out_Files\STARTUP.obj (?C_STARTUP)
         COMMENT TYPE 1: A51 / ASM51 Assembler
  .\Out_Files\system_um800x.obj (SYSTEM_UM800X)
         COMMENT TYPE 0: C51 V9.60.0.0
  .\Out_Files\common.obj (COMMON)
         COMMENT TYPE 0: C51 V9.60.0.0
  .\Out_Files\uart0.obj (UART0)
         COMMENT TYPE 0: C51 V9.60.0.0
  .\Out_Files\adc.obj (ADC)
         COMMENT TYPE 0: C51 V9.60.0.0
  .\Out_Files\app.obj (APP)
         COMMENT TYPE 0: C51 V9.60.0.0
  .\Out_Files\main.obj (MAIN)
         COMMENT TYPE 0: C51 V9.60.0.0
  D:\KEILC51\C51\LIB\C51FPC.LIB (?C?FPMUL)
         COMMENT TYPE 1: A51 / ASM51 Assembler
  D:\KEILC51\C51\LIB\C51FPC.LIB (?C?FPDIV)
         COMMENT TYPE 1: A51 / ASM51 Assembler
  D:\KEILC51\C51\LIB\C51FPC.LIB (?C?FCAST)
         COMMENT TYPE 1: A51 / ASM51 Assembler
  D:\KEILC51\C51\LIB\C51FPC.LIB (PRINTF)
         COMMENT TYPE 1: A51 / ASM51 Assembler
  D:\KEILC51\C51\LIB\C51FPC.LIB (?C?FPGETOPN)
         COMMENT TYPE 1: A51 / ASM51 Assembler
  D:\KEILC51\C51\LIB\C51FPC.LIB (?C?FPROUND)
         COMMENT TYPE 1: A51 / ASM51 Assembler
  D:\KEILC51\C51\LIB\C51FPC.LIB (?C?FPCONVERT)
         COMMENT TYPE 1: A51 / ASM51 Assembler
  D:\KEILC51\C51\LIB\C51FPC.LIB (?C?FPADD)
         COMMENT TYPE 1: A51 / ASM51 Assembler
  D:\KEILC51\C51\LIB\C51FPC.LIB (?C?FTNPWR)
         COMMENT TYPE 1: A51 / ASM51 Assembler
  D:\KEILC51\C51\LIB\C51C.LIB (?C_INIT)
         COMMENT TYPE 1: A51 / ASM51 Assembler
  D:\KEILC51\C51\LIB\C51C.LIB (?C?CLDPTR)
         COMMENT TYPE 1: A51 / ASM51 Assembler
  D:\KEILC51\C51\LIB\C51C.LIB (?C?CLDOPTR)
         COMMENT TYPE 1: A51 / ASM51 Assembler
  D:\KEILC51\C51\LIB\C51C.LIB (?C?CSTPTR)
         COMMENT TYPE 1: A51 / ASM51 Assembler
  D:\KEILC51\C51\LIB\C51C.LIB (?C?LADD)
         COMMENT TYPE 1: A51 / ASM51 Assembler
  D:\KEILC51\C51\LIB\C51C.LIB (?C?LMUL)
         COMMENT TYPE 1: A51 / ASM51 Assembler
  D:\KEILC51\C51\LIB\C51C.LIB (?C?ULDIV)
         COMMENT TYPE 1: A51 / ASM51 Assembler
  D:\KEILC51\C51\LIB\C51C.LIB (?C?LNEG)
         COMMENT TYPE 1: A51 / ASM51 Assembler
  D:\KEILC51\C51\LIB\C51C.LIB (?C?ULCMP)
         COMMENT TYPE 1: A51 / ASM51 Assembler
  D:\KEILC51\C51\LIB\C51C.LIB (?C?ULSHR)
         COMMENT TYPE 1: A51 / ASM51 Assembler
  D:\KEILC51\C51\LIB\C51C.LIB (?C?LLDOPTR)
         COMMENT TYPE 1: A51 / ASM51 Assembler
LX51 LINKER/LOCATER V4.66.97.0                                                        03/02/2021  17:27:53  PAGE 2


  D:\KEILC51\C51\LIB\C51C.LIB (?C?LLDPDATA)
         COMMENT TYPE 1: A51 / ASM51 Assembler
  D:\KEILC51\C51\LIB\C51C.LIB (?C?LLDPDATA0)
         COMMENT TYPE 1: A51 / ASM51 Assembler
  D:\KEILC51\C51\LIB\C51C.LIB (?C?LLDIPDATA)
         COMMENT TYPE 1: A51 / ASM51 Assembler
  D:\KEILC51\C51\LIB\C51C.LIB (?C?LSTPDATA)
         COMMENT TYPE 1: A51 / ASM51 Assembler
  D:\KEILC51\C51\LIB\C51C.LIB (?C?LSTKPDATA)
         COMMENT TYPE 1: A51 / ASM51 Assembler
  D:\KEILC51\C51\LIB\C51C.LIB (?C?PLDPDATA)
         COMMENT TYPE 1: A51 / ASM51 Assembler
  D:\KEILC51\C51\LIB\C51C.LIB (?C?PLDIPDATA)
         COMMENT TYPE 1: A51 / ASM51 Assembler
  D:\KEILC51\C51\LIB\C51C.LIB (?C?PSTPDATA)
         COMMENT TYPE 1: A51 / ASM51 Assembler
  D:\KEILC51\C51\LIB\C51C.LIB (?C?CCASE)
         COMMENT TYPE 1: A51 / ASM51 Assembler
  D:\KEILC51\C51\LIB\C51C.LIB (?C?ICALL)
         COMMENT TYPE 1: A51 / ASM51 Assembler
  D:\KEILC51\C51\LIB\C51C.LIB (?C?DPSEL)
         COMMENT TYPE 1: A51 / ASM51 Assembler
  D:\KEILC51\C51\LIB\C51C.LIB (?C?LLDIDATA)
         COMMENT TYPE 1: A51 / ASM51 Assembler
  D:\KEILC51\C51\LIB\C51C.LIB (?C?LLDXDATA)
         COMMENT TYPE 1: A51 / ASM51 Assembler
  D:\KEILC51\C51\LIB\C51C.LIB (?C?LLDCODE)
         COMMENT TYPE 1: A51 / ASM51 Assembler


ACTIVE MEMORY CLASSES OF MODULE:  .\Out_Files\adc (?C_STARTUP)

BASE        START       END         USED      MEMORY CLASS
==========================================================
X:000000H   X:000000H   X:0007FFH             XDATA
X:000000H   X:000000H   X:0007FFH             HDATA
C:000000H   C:000000H   C:007FFFH   00103DH   CODE
C:000000H   C:000000H   C:007FFFH   00008EH   CONST
C:000000H   C:000000H   C:007FFFH             ECODE
C:000000H   C:000000H   C:007FFFH             HCONST
I:000000H   I:000000H   I:0000FFH   000001H   IDATA
X:000000H   X:000000H   X:0000FFH   0000C1H   PDATA
I:000000H   I:000000H   I:00007FH   00000DH   DATA
I:000020H.0 I:000020H.0 I:00002FH.7 000001H.1 BIT


MEMORY MAP OF MODULE:  .\Out_Files\adc (?C_STARTUP)


START     STOP      LENGTH    ALIGN  RELOC    MEMORY CLASS   SEGMENT NAME
=========================================================================

* * * * * * * * * * *   D A T A   M E M O R Y   * * * * * * * * * * * * *
000000H   000007H   000008H   ---    AT..     DATA           "REG BANK 0"
000008H   00000CH   000005H   BYTE   UNIT     DATA           _DATA_GROUP_
00000DH.0 00001FH.7 000013H.0 ---    ---      **GAP**
000020H.0 000021H.0 000001H.1 BIT    UNIT     BIT            _BIT_GROUP_
000021H.1 000021H   000000H.7 ---    ---      **GAP**
000022H   000022H   000001H   BYTE   UNIT     IDATA          ?STACK

* * * * * * * * * * *   C O D E   M E M O R Y   * * * * * * * * * * * * *
000000H   000002H   000003H   ---    OFFS..   CODE           ?CO??C_STARTUP?0
000003H   000020H   00001EH   BYTE   UNIT     CODE           ?PR?UART0_REC_PRO?APP
000021H   000022H   000002H   ---    ---      **GAP**
000023H   000025H   000003H   BYTE   OFFS..   CODE           ?UART0?00023
LX51 LINKER/LOCATER V4.66.97.0                                                        03/02/2021  17:27:53  PAGE 3


000026H   000030H   00000BH   BYTE   UNIT     CODE           ?PR?SYSTEMINIT?SYSTEM_UM800X
000031H   000032H   000002H   ---    ---      **GAP**
000033H   000035H   000003H   BYTE   OFFS..   CODE           ?ADC?00033
000036H   0007B5H   000780H   BYTE   UNIT     CODE           ?C?LIB_CODE
0007B6H   000C23H   00046EH   BYTE   UNIT     CODE           ?PR?PRINTF?PRINTF
000C24H   000CAFH   00008CH   BYTE   UNIT     CODE           ?C_C51STARTUP
000CB0H   000D24H   000075H   BYTE   UNIT     CODE           ?PR?ADC_SINGLE_MODE_TEST?APP
000D25H   000D94H   000070H   BYTE   UNIT     CODE           ?PR?_UART0_SET_BAUD_RATE?UART0
000D95H   000DFDH   000069H   BYTE   UNIT     CODE           ?PR?ADC_IRQHANDLER?ADC
000DFEH   000E60H   000063H   BYTE   UNIT     CODE           ?PR?UART0_IRQHANDLER?UART0
000E61H   000EB8H   000058H   BYTE   UNIT     CODE           ?PR?_ADC_INIT?ADC
000EB9H   000EFAH   000042H   BYTE   UNIT     CODE           ?PR?_UART0_INIT?UART0
000EFBH   000F3BH   000041H   BYTE   UNIT     CODE           ?PR?_DELAY1MS?COMMON
000F3CH   000F64H   000029H   BYTE   UNIT     CODE           ?C_INITSEG
000F65H   000F8AH   000026H   BYTE   UNIT     CODE           ?PR?_CLOCK_INIT?SYSTEM_UM800X
000F8BH   000FABH   000021H   BYTE   UNIT     CODE           ?PR?UART_INIT?APP
000FACH   000FC8H   00001DH   BYTE   UNIT     CODE           ?PR?_UART0_IRQ_INIT?UART0
000FC9H   000FDEH   000016H   BYTE   UNIT     CODE           ?PR?_UART0_SEND_BYTE?UART0
000FDFH   000FF4H   000016H   BYTE   UNIT     CODE           ?PR?ADC_TEST?APP
000FF5H   001003H   00000FH   BYTE   UNIT     CODE           ?PR?_GET_ADC?ADC
001004H   001011H   00000EH   BYTE   UNIT     CODE           ?PR?_ADC_IO_CONFIG?ADC
001012H   00101FH   00000EH   BYTE   UNIT     CODE           ?PR?_ADC_CONVERT_START?ADC
001020H   00102AH   00000BH   BYTE   UNIT     CODE           ?PR?MAIN?MAIN
00102BH   001032H   000008H   BYTE   UNIT     CODE           ?PR?GET_ADC_VALUE?ADC
001033H   001038H   000006H   BYTE   UNIT     CODE           ?PR?UART0_SEND_PRO?APP
001039H   00103DH   000005H   BYTE   UNIT     CODE           ?PR?_PUTCHAR?UART0
00103EH   001040H   000003H   BYTE   UNIT     CODE           ?PR?UART0_RECV_BYTE?UART0
001041H   0010CEH   00008EH   BYTE   UNIT     CONST          ?CO?APP

* * * * * * * * * * *  X D A T A   M E M O R Y  * * * * * * * * * * * * *
000000H   000098H   000099H   BYTE   INPAGE   PDATA          ?PD?APP
000099H   0000B2H   00001AH   BYTE   INPAGE   PDATA          _PDATA_GROUP_
0000B3H   0000B9H   000007H   BYTE   INPAGE   PDATA          ?PD?UART0
0000BAH   0000BDH   000004H   BYTE   INPAGE   PDATA          ?PD?SYSTEM_UM800X
0000BEH   0000C0H   000003H   BYTE   INPAGE   PDATA          ?PD?ADC

* * * * * * * * *   R E M O V E D     S E G M E N T S   * * * * * * * *
   *DEL*:           000013H   BYTE   UNIT     CODE           ?PR?_DELAY?COMMON
   *DEL*:           000004H   BYTE   INPAGE   PDATA          ?PD?_DELAY?COMMON
   *DEL*:           000062H   BYTE   UNIT     CODE           ?PR?_PRINTF_BUFF_BYTE?COMMON
   *DEL*:           00000BH   BYTE   INPAGE   PDATA          ?PD?_PRINTF_BUFF_BYTE?COMMON
   *DEL*:           00006DH   BYTE   UNIT     CODE           ?PR?_PRINTF_BUFF_WORD?COMMON
   *DEL*:           00000BH   BYTE   INPAGE   PDATA          ?PD?_PRINTF_BUFF_WORD?COMMON
   *DEL*:           000010H   BYTE   UNIT     CONST          ?CO?COMMON
   *DEL*:           00002AH   BYTE   UNIT     CODE           ?PR?_UART0_SEND_BYTES?UART0
   *DEL*:           000007H   BYTE   INPAGE   PDATA          ?PD?_UART0_SEND_BYTES?UART0
   *DEL*:           000007H   BYTE   UNIT     CODE           ?PR?ADC_DEINIT?ADC
   *DEL*:           000018H   BYTE   UNIT     CODE           ?PR?_ADC_IRQ_CONFIG?ADC
   *DEL*:           000007H   BYTE   UNIT     CODE           ?PR?ADC_CONVERT_STOP?ADC
   *DEL*:           000010H   BYTE   UNIT     CODE           ?PR?ADC_SINGLE_MODE_FUNC?APP
   *DEL*:           00001EH   BYTE   UNIT     CODE           ?PR?ADC_CONTINOUS_MODE_FUNC?APP
   *DEL*:           00005BH   BYTE   UNIT     CODE           ?PR?ADC_CONTINOUS_MODE_TEST?APP
   *DEL*:           000001H   BYTE   INPAGE   PDATA          ?PD?ADC_CONTINOUS_MODE_TEST?APP



OVERLAY MAP OF MODULE:   .\Out_Files\adc (?C_STARTUP)


FUNCTION/MODULE                   BIT_GROUP   DATA_GROUP   PDATA_GROUP
--> CALLED FUNCTION/MODULE       START  STOP  START  STOP  START  STOP
======================================================================
?C_C51STARTUP                    ----- -----  ----- -----  ----- -----
  +--> MAIN/MAIN
  +--> ?C_INITSEG
LX51 LINKER/LOCATER V4.66.97.0                                                        03/02/2021  17:27:53  PAGE 4



MAIN/MAIN                        ----- -----  ----- -----  ----- -----
  +--> SYSTEMINIT/SYSTEM_UM800X
  +--> UART_INIT/APP
  +--> ADC_TEST/APP

SYSTEMINIT/SYSTEM_UM800X         ----- -----  ----- -----  ----- -----
  +--> _CLOCK_INIT/SYSTEM_UM800X

_CLOCK_INIT/SYSTEM_UM800X        ----- -----  ----- -----  0099H 009CH

UART_INIT/APP                    ----- -----  ----- -----  ----- -----
  +--> _UART0_INIT/UART0
  +--> UART0_SEND_PRO/APP
  +--> UART0_REC_PRO/APP
  +--> _UART0_IRQ_INIT/UART0

_UART0_INIT/UART0                ----- -----  ----- -----  0099H 009CH
  +--> _UART0_SET_BAUD_RATE/UART0

_UART0_SET_BAUD_RATE/UART0       ----- -----  ----- -----  009DH 00A8H

UART0_SEND_PRO/APP               ----- -----  ----- -----  ----- -----

UART0_REC_PRO/APP                ----- -----  ----- -----  ----- -----
  +--> UART0_RECV_BYTE/UART0

UART0_RECV_BYTE/UART0            ----- -----  ----- -----  ----- -----

_UART0_IRQ_INIT/UART0            ----- -----  ----- -----  0099H 009FH

ADC_TEST/APP                     ----- -----  ----- -----  ----- -----
  +--> PRINTF/PRINTF
  +--> ADC_SINGLE_MODE_TEST/APP

PRINTF/PRINTF                    20H.0 21H.0  0008H 000CH  009CH 00B2H
  +--> _PUTCHAR/UART0

_PUTCHAR/UART0                   ----- -----  ----- -----  ----- -----
  +--> _UART0_SEND_BYTE/UART0

_UART0_SEND_BYTE/UART0           ----- -----  ----- -----  ----- -----

ADC_SINGLE_MODE_TEST/APP         ----- -----  ----- -----  0099H 009BH
  +--> _ADC_INIT/ADC
  +--> _ADC_IO_CONFIG/ADC
  +--> _GET_ADC/ADC
  +--> PRINTF/PRINTF
  +--> _DELAY1MS/COMMON

_ADC_INIT/ADC                    ----- -----  ----- -----  009CH 00A0H

_ADC_IO_CONFIG/ADC               ----- -----  ----- -----  ----- -----

_GET_ADC/ADC                     ----- -----  ----- -----  ----- -----
  +--> _ADC_CONVERT_START/ADC
  +--> GET_ADC_VALUE/ADC

_ADC_CONVERT_START/ADC           ----- -----  ----- -----  ----- -----

GET_ADC_VALUE/ADC                ----- -----  ----- -----  ----- -----

_DELAY1MS/COMMON                 ----- -----  ----- -----  009CH 00A3H

?C_INITSEG                       ----- -----  ----- -----  ----- -----
LX51 LINKER/LOCATER V4.66.97.0                                                        03/02/2021  17:27:53  PAGE 5



*** NEW ROOT *******************

UART0_IRQHANDLER/UART0           ----- -----  ----- -----  ----- -----

*** NEW ROOT *******************

ADC_IRQHANDLER/ADC               ----- -----  ----- -----  ----- -----



PUBLIC SYMBOLS OF MODULE:  .\Out_Files\adc (?C_STARTUP)


      VALUE       CLASS    TYPE      PUBLIC SYMBOL NAME
      =================================================
      0200009CH   PDATA    BYTE      ?_adc_init?BYTE
      0200009CH   PDATA    ---       ?_PRINTF?BYTE
      0200009CH   PDATA    ---       ?_SPRINTF?BYTE
      02000099H   PDATA    BYTE      ?_uart0_irq_init?BYTE
      01000762H   CODE     ---       ?C?CCASE
      01000517H   CODE     ---       ?C?CLDOPTR
      010004FEH   CODE     ---       ?C?CLDPTR
      00000000H   NUMBER   ---       ?C?CODESEG
      01000544H   CODE     ---       ?C?CSTPTR
      00000092H   DATA     ---       ?C?DPSEL
      010001E6H   CODE     ---       ?C?FCASTC
      010001E1H   CODE     ---       ?C?FCASTI
      010001DCH   CODE     ---       ?C?FCASTL
      0100039DH   CODE     ---       ?C?FPADD
      01000293H   CODE     ---       ?C?FPCONVERT
      0100013FH   CODE     ---       ?C?FPDIV
      0100021AH   CODE     ---       ?C?FPGETOPN2
      01000036H   CODE     ---       ?C?FPMUL
      0100024FH   CODE     ---       ?C?FPNANRESULT
      01000259H   CODE     ---       ?C?FPOVERFLOW
      01000231H   CODE     ---       ?C?FPRESULT
      01000245H   CODE     ---       ?C?FPRESULT2
      01000264H   CODE     ---       ?C?FPROUND
      01000399H   CODE     ---       ?C?FPSUB
      01000256H   CODE     ---       ?C?FPUNDERFLOW
      010004BEH   CODE     ---       ?C?FTNPWR
      01000788H   CODE     ---       ?C?ICALL
      0100078CH   CODE     ---       ?C?ICALL2
      01000556H   CODE     ---       ?C?LADD
      010007A6H   CODE     ---       ?C?LLDCODE
      0100078EH   CODE     ---       ?C?LLDIDATA
      01000704H   CODE     ---       ?C?LLDIPDATA
      010006FBH   CODE     ---       ?C?LLDIPDATA1
      010006FDH   CODE     ---       ?C?LLDIPDATA8
      010006B2H   CODE     ---       ?C?LLDOPTR
      010006E2H   CODE     ---       ?C?LLDPDATA
      010006EEH   CODE     ---       ?C?LLDPDATA0
      0100079AH   CODE     ---       ?C?LLDXDATA
      01000563H   CODE     ---       ?C?LMUL
      01000680H   CODE     ---       ?C?LNEG
      01000727H   CODE     ---       ?C?LSTKPDATA
      0100071BH   CODE     ---       ?C?LSTPDATA
      01000749H   CODE     ---       ?C?PLDIPDATA
      01000740H   CODE     ---       ?C?PLDPDATA
      01000759H   CODE     ---       ?C?PSTPDATA
      0100068EH   CODE     ---       ?C?ULCMP
      010005EEH   CODE     ---       ?C?ULDIV
      0100069FH   CODE     ---       ?C?ULSHR
      00000000H   NUMBER   ---       ?C?XDATASEG
LX51 LINKER/LOCATER V4.66.97.0                                                        03/02/2021  17:27:53  PAGE 6


      01000C6BH   CODE     ---       ?C_START
      01000000H   CODE     ---       ?C_STARTUP
      01001012H   CODE     ---       _adc_convert_start
      01000E61H   CODE     ---       _adc_init
      01001004H   CODE     ---       _adc_io_config
*DEL*:00000000H   CODE     ---       _adc_irq_config
      01000F65H   CODE     ---       _clock_init
*DEL*:00000000H   CODE     ---       _delay
      01000EFBH   CODE     ---       _delay1ms
      01000FF5H   CODE     ---       _get_adc
      01000818H   CODE     ---       _PRINTF
*DEL*:00000000H   CODE     ---       _printf_buff_byte
*DEL*:00000000H   CODE     ---       _printf_buff_word
      01001039H   CODE     ---       _putchar
      01000812H   CODE     ---       _SPRINTF
      01000EB9H   CODE     ---       _uart0_init
      01000FACH   CODE     ---       _uart0_irq_init
      01000FC9H   CODE     ---       _uart0_send_byte
*DEL*:00000000H   CODE     ---       _uart0_send_bytes
*SFR* 000000D0H.6 DATA     BIT       AC
*SFR* 000000E0H   DATA     BYTE      ACC
*SFR* 000000E0H.0 DATA     BIT       ACC0
*SFR* 000000E0H.1 DATA     BIT       ACC1
*SFR* 000000E0H.2 DATA     BIT       ACC2
*SFR* 000000E0H.3 DATA     BIT       ACC3
*SFR* 000000E0H.4 DATA     BIT       ACC4
*SFR* 000000E0H.5 DATA     BIT       ACC5
*SFR* 000000E0H.6 DATA     BIT       ACC6
*SFR* 000000E0H.7 DATA     BIT       ACC7
*DEL*:00000000H   CODE     ---       adc_continous_mode_func
*DEL*:00000000H   CODE     ---       adc_continous_mode_test
*DEL*:00000000H   CODE     ---       adc_convert_stop
      02000001H   PDATA    ---       adc_converte_val
      02000051H   PDATA    WORD      adc_data
*DEL*:00000000H   CODE     ---       adc_deinit
      01000D95H   CODE     ---       ADC_IRQHandler
      02000000H   PDATA    BYTE      adc_rx_count
      02000094H   PDATA    BYTE      adc_rx_flag
*DEL*:00000000H   CODE     ---       adc_single_mode_func
      01000CB0H   CODE     ---       adc_single_mode_test
      01000FDFH   CODE     ---       adc_test
*SFR* 000000FEH   DATA     BYTE      ADCCDR0
*SFR* 000000FFH   DATA     BYTE      ADCCDR1
*SFR* 000000EDH   DATA     BYTE      ADCCONT
*SFR* 000000F6H   DATA     BYTE      ADCCSTAT
*SFR* 000000B6H   DATA     WORD      ADCDR
*SFR* 000000B6H   DATA     BYTE      ADCDR0
*SFR* 000000B7H   DATA     BYTE      ADCDR1
      020000BEH   PDATA    ---       adcfunc
*SFR* 000000ACH   DATA     BYTE      ADCGCR0
*SFR* 000000ADH   DATA     BYTE      ADCGCR1
*SFR* 000000B4H   DATA     BYTE      ADCGCR2
*SFR* 000000B5H   DATA     BYTE      ADCGCR3
*SFR* 000000F5H   DATA     BYTE      ADCHL
*SFR* 00000093H   DATA     BYTE      ADCIER
*SFR* 000000F7H   DATA     BYTE      ADCSPW
*SFR* 000000FDH   DATA     BYTE      ADCVREF
*SFR* 000000F0H   DATA     BYTE      B
*SFR* 000000F0H.0 DATA     BIT       B0
*SFR* 000000F0H.1 DATA     BIT       B1
*SFR* 000000F0H.2 DATA     BIT       B2
*SFR* 000000F0H.3 DATA     BIT       B3
*SFR* 000000F0H.4 DATA     BIT       B4
*SFR* 000000F0H.5 DATA     BIT       B5
*SFR* 000000F0H.6 DATA     BIT       B6
LX51 LINKER/LOCATER V4.66.97.0                                                        03/02/2021  17:27:53  PAGE 7


*SFR* 000000F0H.7 DATA     BIT       B7
*SFR* 00000086H   DATA     BYTE      BEEPCTR
*SFR* 000000F8H   DATA     BYTE      CLKCON
*SFR* 000000B1H   DATA     BYTE      CLKST
*SFR* 000000D0H.7 DATA     BIT       CY
*SFR* 00000095H   DATA     BYTE      D_PAGESEL
*SFR* 00000083H   DATA     BYTE      DPH
*SFR* 00000085H   DATA     BYTE      DPH1
*SFR* 00000082H   DATA     BYTE      DPL
*SFR* 00000084H   DATA     BYTE      DPL1
*SFR* 00000092H   DATA     BYTE      DPS
*SFR* 000000A8H.7 DATA     BIT       EA
*SFR* 000000A8H.6 DATA     BIT       EADC
*SFR* 000000B8H.3 DATA     BIT       EFCINTEN
*SFR* 000000A8H.5 DATA     BIT       EPWM
*SFR* 000000D8H.3 DATA     BIT       ERSTF
*SFR* 000000A8H.4 DATA     BIT       ES0
*SFR* 000000A8H.2 DATA     BIT       ES1
*SFR* 000000B2H   DATA     BYTE      ESTCR
*SFR* 000000A8H.1 DATA     BIT       ET0
*SFR* 000000A8H.3 DATA     BIT       ET1
*SFR* 0000009EH   DATA     BYTE      EUARTEN
*SFR* 000000A8H.0 DATA     BIT       EX0
*SFR* 000000D0H.5 DATA     BIT       F0
*SFR* 000000D0H.1 DATA     BIT       F1
      0100102BH   CODE     ---       get_adc_value
*SFR* 000000A8H   DATA     BYTE      IEN0
*SFR* 000000B8H   DATA     BYTE      IEN1
*SFR* 000000A9H   DATA     BYTE      IP0
*SFR* 000000B9H   DATA     BYTE      IP1
*SFR* 000000BDH   DATA     BYTE      LDOTRIMH
*SFR* 00000091H   DATA     BYTE      LDOTRIML
*SFR* 000000DDH   DATA     BYTE      LVDCON
*SFR* 000000D8H.5 DATA     BIT       LVRF
      01001020H   CODE     ---       main
*SFR* 000000D1H   DATA     WORD      OADR
*SFR* 000000D2H   DATA     BYTE      OADRH
*SFR* 000000D1H   DATA     BYTE      OADRL
*SFR* 000000D4H   DATA     BYTE      OCTRL
*SFR* 000000D3H   DATA     BYTE      ODATA
*SFR* 000000A2H   DATA     BYTE      OINTEN
*SFR* 000000A3H   DATA     BYTE      OINTUS
*SFR* 000000A7H   DATA     BYTE      OPSET
*SFR* 000000A6H   DATA     BYTE      OSTATUS
*SFR* 000000A1H   DATA     BYTE      OUS
*SFR* 000000D0H.0 DATA     BIT       P
*SFR* 00000080H   DATA     BYTE      P0
*SFR* 00000080H.0 DATA     BIT       P00
*SFR* 00000080H.1 DATA     BIT       P01
*SFR* 00000080H.2 DATA     BIT       P02
*SFR* 00000080H.3 DATA     BIT       P03
*SFR* 00000080H.4 DATA     BIT       P04
*SFR* 000000D7H   DATA     BYTE      P0CS
*SFR* 00000097H   DATA     BYTE      P0DR
*SFR* 000000E9H   DATA     BYTE      P0IEN
*SFR* 000000E1H   DATA     BYTE      P0IRQ
*SFR* 000000D6H   DATA     BYTE      P0OD
*SFR* 000000F9H   DATA     BYTE      P0OEN
*SFR* 000000D5H   DATA     BYTE      P0PD
*SFR* 000000F1H   DATA     BYTE      P0PU
*SFR* 00000090H   DATA     BYTE      P1
*SFR* 00000090H.0 DATA     BIT       P10
*SFR* 00000090H.1 DATA     BIT       P11
*SFR* 00000090H.2 DATA     BIT       P12
*SFR* 00000090H.3 DATA     BIT       P13
LX51 LINKER/LOCATER V4.66.97.0                                                        03/02/2021  17:27:53  PAGE 8


*SFR* 00000090H.4 DATA     BIT       P14
*SFR* 00000090H.5 DATA     BIT       P15
*SFR* 000000DCH   DATA     BYTE      P1CS
*SFR* 000000E5H   DATA     BYTE      P1DR
*SFR* 000000EAH   DATA     BYTE      P1IEN
*SFR* 000000E2H   DATA     BYTE      P1IRQ
*SFR* 000000DBH   DATA     BYTE      P1OD
*SFR* 000000FAH   DATA     BYTE      P1OEN
*SFR* 000000DAH   DATA     BYTE      P1PD
*SFR* 000000F2H   DATA     BYTE      P1PU
*SFR* 000000A0H   DATA     BYTE      P2
*SFR* 000000A0H.0 DATA     BIT       P20
*SFR* 000000A0H.2 DATA     BIT       P22
*SFR* 000000A0H.3 DATA     BIT       P23
*SFR* 000000A0H.5 DATA     BIT       P25
*SFR* 000000A0H.6 DATA     BIT       P26
*SFR* 000000A0H.7 DATA     BIT       P27
*SFR* 000000F4H   DATA     BYTE      P2CS
*SFR* 000000FCH   DATA     BYTE      P2DR
*SFR* 000000EBH   DATA     BYTE      P2IEN
*SFR* 000000E3H   DATA     BYTE      P2IRQ
*SFR* 000000ECH   DATA     BYTE      P2OD
*SFR* 000000FBH   DATA     BYTE      P2OEN
*SFR* 000000E4H   DATA     BYTE      P2PD
*SFR* 000000F3H   DATA     BYTE      P2PU
*SFR* 00000094H   DATA     BYTE      PAGESEL
*SFR* 000000DEH   DATA     BYTE      PCLK0
*SFR* 000000DFH   DATA     BYTE      PCLK1
*SFR* 00000087H   DATA     BYTE      PCON
*SFR* 0000008EH   DATA     BYTE      PDSEL
*SFR* 0000008FH   DATA     BYTE      POREN
*SFR* 000000D8H.4 DATA     BIT       PORF
*SFR* 000000E6H   DATA     BYTE      PRESET0
*SFR* 000000E7H   DATA     BYTE      PRESET1
*SFR* 000000D0H   DATA     BYTE      PSW
*SFR* 000000C8H   DATA     BYTE      PWM0CON
*SFR* 000000C4H   DATA     BYTE      PWM0DH
*SFR* 000000C3H   DATA     BYTE      PWM0DL
*SFR* 000000C8H.7 DATA     BIT       PWM0EN
*SFR* 000000C8H.2 DATA     BIT       PWM0IE
*SFR* 000000C8H.1 DATA     BIT       PWM0IF
*SFR* 000000CCH   DATA     BYTE      PWM0PH
*SFR* 000000CBH   DATA     BYTE      PWM0PL
*SFR* 000000C8H.6 DATA     BIT       PWM0S
*SFR* 000000C8H.0 DATA     BIT       PWM0SS
*SFR* 000000C9H   DATA     BYTE      PWM1CON
*SFR* 000000C6H   DATA     BYTE      PWM1DH
*SFR* 000000C5H   DATA     BYTE      PWM1DL
*SFR* 000000CEH   DATA     BYTE      PWM1PH
*SFR* 000000CDH   DATA     BYTE      PWM1PL
*SFR* 000000CAH   DATA     BYTE      PWM2CON
*SFR* 000000C7H   DATA     BYTE      PWM2DH
*SFR* 000000CFH   DATA     BYTE      PWM2DL
*SFR* 000000C2H   DATA     BYTE      PWM2PH
*SFR* 000000C1H   DATA     BYTE      PWM2PL
*SFR* 00000098H.2 DATA     BIT       RB80
*SFR* 000000F8H.2 DATA     BIT       RC16MEN
*SFR* 000000F8H.5 DATA     BIT       RC16MF
*SFR* 000000F8H.3 DATA     BIT       RC32KEN
*SFR* 000000F8H.6 DATA     BIT       RC32KF
*SFR* 000000EEH   DATA     BYTE      RCHDIV
*SFR* 000000BEH   DATA     BYTE      RCHTRIMH
*SFR* 000000BFH   DATA     BYTE      RCHTRIML
*SFR* 0000009FH   DATA     BYTE      RCLTRIM
*SFR* 000000AFH   DATA     BYTE      REMAP
LX51 LINKER/LOCATER V4.66.97.0                                                        03/02/2021  17:27:53  PAGE 9


*SFR* 00000098H.4 DATA     BIT       REN0
*SFR* 00000098H.0 DATA     BIT       RI0
*SFR* 000000D0H.3 DATA     BIT       RS0
*SFR* 000000D0H.4 DATA     BIT       RS1
*SFR* 000000D8H   DATA     BYTE      RSTSTAT
      02000095H   PDATA    WORD      rx_count
      02000093H   PDATA    BYTE      rx_flag
*SFR* 00000099H   DATA     BYTE      S0BUF
*SFR* 00000098H   DATA     BYTE      S0CON
*SFR* 000000BAH   DATA     BYTE      S0RELH
*SFR* 000000AAH   DATA     BYTE      S0RELL
*SFR* 0000009CH   DATA     BYTE      S1BUF
*SFR* 0000009BH   DATA     BYTE      S1CON
*SFR* 000000BBH   DATA     BYTE      S1RELH
*SFR* 0000009DH   DATA     BYTE      S1RELL
*SFR* 00000098H.7 DATA     BIT       SM0
*SFR* 00000098H.6 DATA     BIT       SM1
*SFR* 00000098H.5 DATA     BIT       SM20
*SFR* 00000081H   DATA     BYTE      SP
*SFR* 000000B8H.1 DATA     BIT       SPIINTEN
*SFR* 000000D9H   DATA     BYTE      SYSDIV
*SFR* 000000F8H.0 DATA     BIT       SYSSEL
      020000BAH   PDATA    DWORD     SystemCoreClock
      01000026H   CODE     ---       systeminit
*SFR* 00000088H.0 DATA     BIT       T0CLKS
*SFR* 00000088H.4 DATA     BIT       T1CLKS
*SFR* 000000ABH   DATA     BYTE      T2CON
*SFR* 00000098H.3 DATA     BIT       TB80
*SFR* 00000088H   DATA     BYTE      TCON
*SFR* 00000088H.3 DATA     BIT       TF0
*SFR* 00000088H.7 DATA     BIT       TF1
*SFR* 0000008CH   DATA     BYTE      TH0
*SFR* 0000008DH   DATA     BYTE      TH1
*SFR* 00000098H.1 DATA     BIT       TI0
*SFR* 0000008AH   DATA     BYTE      TL0
*SFR* 0000008BH   DATA     BYTE      TL1
*SFR* 00000089H   DATA     BYTE      TMOD
*SFR* 00000088H.1 DATA     BIT       TR0
*SFR* 00000088H.5 DATA     BIT       TR1
      02000097H   PDATA    WORD      tx_count
      020000B9H   PDATA    BYTE      tx_flag
      01000DFEH   CODE     ---       UART0_IRQHandler
      01000003H   CODE     ---       uart0_rec_pro
      0100103EH   CODE     ---       uart0_recv_byte
      02000053H   PDATA    ---       uart0_rx_buf
      01001033H   CODE     ---       uart0_send_pro
      02000073H   PDATA    ---       uart0_tx_buf
      020000B3H   PDATA    ---       uart0func
      01000F8BH   CODE     ---       uart_init
*SFR* 000000D8H.6 DATA     BIT       WDEN
*SFR* 000000D8H.7 DATA     BIT       WDOF
*SFR* 000000D8H.0 DATA     BIT       WDT0
*SFR* 000000D8H.1 DATA     BIT       WDT1
*SFR* 000000D8H.2 DATA     BIT       WDT2
*SFR* 000000F8H.1 DATA     BIT       XCLKEN
*SFR* 000000F8H.4 DATA     BIT       XCLKF
*SFR* 000000B3H   DATA     BYTE      XTHCTR



SYMBOL TABLE OF MODULE:  .\Out_Files\adc (?C_STARTUP)

      VALUE       REP       CLASS    TYPE      SYMBOL NAME
      ====================================================
      ---         MODULE    ---      ---       ?C_STARTUP
LX51 LINKER/LOCATER V4.66.97.0                                                        03/02/2021  17:27:53  PAGE 10


      01000000H   PUBLIC    CODE     ---       ?C_STARTUP
      000000E0H   SYMBOL    DATA     ---       ACC
      000000F0H   SYMBOL    DATA     ---       B
      00000083H   SYMBOL    DATA     ---       DPH
      00000082H   SYMBOL    DATA     ---       DPL
      00000000H   SYMBOL    NUMBER   ---       IBPSTACK
      00000100H   SYMBOL    NUMBER   ---       IBPSTACKTOP
      00000080H   SYMBOL    NUMBER   ---       IDATALEN
      01000C27H   SYMBOL    CODE     ---       IDATALOOP
      00000000H   SYMBOL    NUMBER   ---       PBPSTACK
      00000100H   SYMBOL    NUMBER   ---       PBPSTACKTOP
      00000000H   SYMBOL    NUMBER   ---       PDATALEN
      00000000H   SYMBOL    NUMBER   ---       PDATASTART
      00000000H   SYMBOL    NUMBER   ---       PPAGE
      00000000H   SYMBOL    NUMBER   ---       PPAGEENABLE
      000000A0H   SYMBOL    DATA     ---       PPAGE_SFR
      00000081H   SYMBOL    DATA     ---       SP
      01000C24H   SYMBOL    CODE     ---       STARTUP1
      00000000H   SYMBOL    NUMBER   ---       XBPSTACK
      00000000H   SYMBOL    NUMBER   ---       XBPSTACKTOP
      00000000H   SYMBOL    NUMBER   ---       XDATALEN
      00000000H   SYMBOL    NUMBER   ---       XDATASTART
      01000000H   LINE      CODE     ---       #126
      01000C24H   LINE      CODE     ---       #134
      01000C26H   LINE      CODE     ---       #135
      01000C27H   LINE      CODE     ---       #136
      01000C28H   LINE      CODE     ---       #137
      01000C2AH   LINE      CODE     ---       #191
      01000C2DH   LINE      CODE     ---       #205

      ---         MODULE    ---      ---       SYSTEM_UM800X
      020000BAH   PUBLIC    PDATA    DWORD     SystemCoreClock
      01000026H   PUBLIC    CODE     ---       systeminit
      01000F65H   PUBLIC    CODE     ---       _clock_init
      00000098H.3 SFRSYM    DATA     BIT       TB80
      000000EDH   SFRSYM    DATA     BYTE      ADCCONT
      000000E0H.7 SFRSYM    DATA     BIT       ACC7
      00000080H   SFRSYM    DATA     BYTE      P0
      00000090H   SFRSYM    DATA     BYTE      P1
      000000A0H   SFRSYM    DATA     BYTE      P2
      00000098H.5 SFRSYM    DATA     BIT       SM20
      000000B2H   SFRSYM    DATA     BYTE      ESTCR
      000000B1H   SFRSYM    DATA     BYTE      CLKST
      000000D0H.6 SFRSYM    DATA     BIT       AC
      00000094H   SFRSYM    DATA     BYTE      PAGESEL
      000000D8H.3 SFRSYM    DATA     BIT       ERSTF
      000000E6H   SFRSYM    DATA     BYTE      PRESET0
      000000D4H   SFRSYM    DATA     BYTE      OCTRL
      000000A8H.7 SFRSYM    DATA     BIT       EA
      0000008FH   SFRSYM    DATA     BYTE      POREN
      000000C8H   SFRSYM    DATA     BYTE      PWM0CON
      000000E7H   SFRSYM    DATA     BYTE      PRESET1
      000000C9H   SFRSYM    DATA     BYTE      PWM1CON
      00000086H   SFRSYM    DATA     BYTE      BEEPCTR
      000000CAH   SFRSYM    DATA     BYTE      PWM2CON
      000000F8H.6 SFRSYM    DATA     BIT       RC32KF
      000000A8H   SFRSYM    DATA     BYTE      IEN0
      000000A7H   SFRSYM    DATA     BYTE      OPSET
      000000B8H   SFRSYM    DATA     BYTE      IEN1
      000000A8H.6 SFRSYM    DATA     BIT       EADC
      00000085H   SFRSYM    DATA     BYTE      DPH1
      000000B6H   SFRSYM    DATA     BYTE      ADCDR0
      000000F8H.5 SFRSYM    DATA     BIT       RC16MF
      000000B7H   SFRSYM    DATA     BYTE      ADCDR1
      00000084H   SFRSYM    DATA     BYTE      DPL1
LX51 LINKER/LOCATER V4.66.97.0                                                        03/02/2021  17:27:53  PAGE 11


      000000D6H   SFRSYM    DATA     BYTE      P0OD
      000000DBH   SFRSYM    DATA     BYTE      P1OD
      000000D5H   SFRSYM    DATA     BYTE      P0PD
      00000098H.4 SFRSYM    DATA     BIT       REN0
      000000ECH   SFRSYM    DATA     BYTE      P2OD
      000000DAH   SFRSYM    DATA     BYTE      P1PD
      000000E4H   SFRSYM    DATA     BYTE      P2PD
      000000D7H   SFRSYM    DATA     BYTE      P0CS
      00000097H   SFRSYM    DATA     BYTE      P0DR
      0000009EH   SFRSYM    DATA     BYTE      EUARTEN
      000000DCH   SFRSYM    DATA     BYTE      P1CS
      000000E5H   SFRSYM    DATA     BYTE      P1DR
      000000F4H   SFRSYM    DATA     BYTE      P2CS
      000000FCH   SFRSYM    DATA     BYTE      P2DR
      000000D0H.7 SFRSYM    DATA     BIT       CY
      000000D8H.0 SFRSYM    DATA     BIT       WDT0
      0000009FH   SFRSYM    DATA     BYTE      RCLTRIM
      000000D8H.1 SFRSYM    DATA     BIT       WDT1
      000000D8H.2 SFRSYM    DATA     BIT       WDT2
      00000081H   SFRSYM    DATA     BYTE      SP
      000000F1H   SFRSYM    DATA     BYTE      P0PU
      000000F2H   SFRSYM    DATA     BYTE      P1PU
      000000D1H   SFRSYM    DATA     WORD      OADR
      000000F3H   SFRSYM    DATA     BYTE      P2PU
      00000095H   SFRSYM    DATA     BYTE      D_PAGESEL
      00000093H   SFRSYM    DATA     BYTE      ADCIER
      000000D8H.6 SFRSYM    DATA     BIT       WDEN
      000000BAH   SFRSYM    DATA     BYTE      S0RELH
      00000080H.0 SFRSYM    DATA     BIT       P00
      000000D8H.7 SFRSYM    DATA     BIT       WDOF
      000000BBH   SFRSYM    DATA     BYTE      S1RELH
      00000090H.0 SFRSYM    DATA     BIT       P10
      00000080H.1 SFRSYM    DATA     BIT       P01
      00000087H   SFRSYM    DATA     BYTE      PCON
      000000C4H   SFRSYM    DATA     BYTE      PWM0DH
      000000A0H.0 SFRSYM    DATA     BIT       P20
      00000090H.1 SFRSYM    DATA     BIT       P11
      00000080H.2 SFRSYM    DATA     BIT       P02
      00000088H.0 SFRSYM    DATA     BIT       T0CLKS
      000000C6H   SFRSYM    DATA     BYTE      PWM1DH
      00000090H.2 SFRSYM    DATA     BIT       P12
      00000080H.3 SFRSYM    DATA     BIT       P03
      00000088H.4 SFRSYM    DATA     BIT       T1CLKS
      000000C7H   SFRSYM    DATA     BYTE      PWM2DH
      000000C8H.2 SFRSYM    DATA     BIT       PWM0IE
      000000AAH   SFRSYM    DATA     BYTE      S0RELL
      000000A0H.2 SFRSYM    DATA     BIT       P22
      00000090H.3 SFRSYM    DATA     BIT       P13
      00000080H.4 SFRSYM    DATA     BIT       P04
      00000089H   SFRSYM    DATA     BYTE      TMOD
      00000088H   SFRSYM    DATA     BYTE      TCON
      000000C8H.1 SFRSYM    DATA     BIT       PWM0IF
      0000009DH   SFRSYM    DATA     BYTE      S1RELL
      000000A0H.3 SFRSYM    DATA     BIT       P23
      00000090H.4 SFRSYM    DATA     BIT       P14
      000000C3H   SFRSYM    DATA     BYTE      PWM0DL
      00000090H.5 SFRSYM    DATA     BIT       P15
      000000A6H   SFRSYM    DATA     BYTE      OSTATUS
      000000C5H   SFRSYM    DATA     BYTE      PWM1DL
      000000A0H.5 SFRSYM    DATA     BIT       P25
      000000D8H.4 SFRSYM    DATA     BIT       PORF
      000000D8H   SFRSYM    DATA     BYTE      RSTSTAT
      000000CFH   SFRSYM    DATA     BYTE      PWM2DL
      000000A0H.6 SFRSYM    DATA     BIT       P26
      000000C8H.7 SFRSYM    DATA     BIT       PWM0EN
LX51 LINKER/LOCATER V4.66.97.0                                                        03/02/2021  17:27:53  PAGE 12


      000000A0H.7 SFRSYM    DATA     BIT       P27
      000000A8H.5 SFRSYM    DATA     BIT       EPWM
      000000D8H.5 SFRSYM    DATA     BIT       LVRF
      000000F8H   SFRSYM    DATA     BYTE      CLKCON
      000000CCH   SFRSYM    DATA     BYTE      PWM0PH
      000000CEH   SFRSYM    DATA     BYTE      PWM1PH
      000000C2H   SFRSYM    DATA     BYTE      PWM2PH
      000000F0H   SFRSYM    DATA     BYTE      B
      000000EEH   SFRSYM    DATA     BYTE      RCHDIV
      000000CBH   SFRSYM    DATA     BYTE      PWM0PL
      000000CDH   SFRSYM    DATA     BYTE      PWM1PL
      000000C1H   SFRSYM    DATA     BYTE      PWM2PL
      000000F7H   SFRSYM    DATA     BYTE      ADCSPW
      000000F8H.1 SFRSYM    DATA     BIT       XCLKEN
      000000E0H   SFRSYM    DATA     BYTE      ACC
      000000DDH   SFRSYM    DATA     BYTE      LVDCON
      000000A8H.4 SFRSYM    DATA     BIT       ES0
      000000A9H   SFRSYM    DATA     BYTE      IP0
      000000A8H.1 SFRSYM    DATA     BIT       ET0
      000000A8H.2 SFRSYM    DATA     BIT       ES1
      00000088H.3 SFRSYM    DATA     BIT       TF0
      000000F6H   SFRSYM    DATA     BYTE      ADCCSTAT
      000000B9H   SFRSYM    DATA     BYTE      IP1
      000000A8H.3 SFRSYM    DATA     BIT       ET1
      00000088H.7 SFRSYM    DATA     BIT       TF1
      00000098H.0 SFRSYM    DATA     BIT       RI0
      0000008CH   SFRSYM    DATA     BYTE      TH0
      000000C8H.0 SFRSYM    DATA     BIT       PWM0SS
      0000008DH   SFRSYM    DATA     BYTE      TH1
      00000098H.1 SFRSYM    DATA     BIT       TI0
      000000A8H.0 SFRSYM    DATA     BIT       EX0
      000000D0H.0 SFRSYM    DATA     BIT       P
      000000B8H.3 SFRSYM    DATA     BIT       EFCINTEN
      000000A2H   SFRSYM    DATA     BYTE      OINTEN
      0000008AH   SFRSYM    DATA     BYTE      TL0
      00000098H.7 SFRSYM    DATA     BIT       SM0
      0000008BH   SFRSYM    DATA     BYTE      TL1
      00000098H.6 SFRSYM    DATA     BIT       SM1
      000000FEH   SFRSYM    DATA     BYTE      ADCCDR0
      000000FFH   SFRSYM    DATA     BYTE      ADCCDR1
      000000D0H.3 SFRSYM    DATA     BIT       RS0
      00000088H.1 SFRSYM    DATA     BIT       TR0
      000000ACH   SFRSYM    DATA     BYTE      ADCGCR0
      000000D0H.4 SFRSYM    DATA     BIT       RS1
      00000088H.5 SFRSYM    DATA     BIT       TR1
      000000ADH   SFRSYM    DATA     BYTE      ADCGCR1
      000000B4H   SFRSYM    DATA     BYTE      ADCGCR2
      000000B5H   SFRSYM    DATA     BYTE      ADCGCR3
      000000F8H.3 SFRSYM    DATA     BIT       RC32KEN
      000000DEH   SFRSYM    DATA     BYTE      PCLK0
      000000DFH   SFRSYM    DATA     BYTE      PCLK1
      00000083H   SFRSYM    DATA     BYTE      DPH
      000000E9H   SFRSYM    DATA     BYTE      P0IEN
      000000F5H   SFRSYM    DATA     BYTE      ADCHL
      000000F8H.2 SFRSYM    DATA     BIT       RC16MEN
      000000EAH   SFRSYM    DATA     BYTE      P1IEN
      000000EBH   SFRSYM    DATA     BYTE      P2IEN
      000000B6H   SFRSYM    DATA     WORD      ADCDR
      000000B3H   SFRSYM    DATA     BYTE      XTHCTR
      00000082H   SFRSYM    DATA     BYTE      DPL
      00000099H   SFRSYM    DATA     BYTE      S0BUF
      0000009CH   SFRSYM    DATA     BYTE      S1BUF
      000000F9H   SFRSYM    DATA     BYTE      P0OEN
      000000D9H   SFRSYM    DATA     BYTE      SYSDIV
      00000098H   SFRSYM    DATA     BYTE      S0CON
LX51 LINKER/LOCATER V4.66.97.0                                                        03/02/2021  17:27:53  PAGE 13


      000000FAH   SFRSYM    DATA     BYTE      P1OEN
      000000A3H   SFRSYM    DATA     BYTE      OINTUS
      000000BEH   SFRSYM    DATA     BYTE      RCHTRIMH
      000000F8H.0 SFRSYM    DATA     BIT       SYSSEL
      0000009BH   SFRSYM    DATA     BYTE      S1CON
      000000FBH   SFRSYM    DATA     BYTE      P2OEN
      000000BDH   SFRSYM    DATA     BYTE      LDOTRIMH
      000000ABH   SFRSYM    DATA     BYTE      T2CON
      00000092H   SFRSYM    DATA     BYTE      DPS
      000000BFH   SFRSYM    DATA     BYTE      RCHTRIML
      000000D3H   SFRSYM    DATA     BYTE      ODATA
      00000091H   SFRSYM    DATA     BYTE      LDOTRIML
      000000E1H   SFRSYM    DATA     BYTE      P0IRQ
      000000B8H.1 SFRSYM    DATA     BIT       SPIINTEN
      000000E2H   SFRSYM    DATA     BYTE      P1IRQ
      000000E3H   SFRSYM    DATA     BYTE      P2IRQ
      000000D2H   SFRSYM    DATA     BYTE      OADRH
      000000F0H.0 SFRSYM    DATA     BIT       B0
      000000F0H.1 SFRSYM    DATA     BIT       B1
      000000F0H.2 SFRSYM    DATA     BIT       B2
      000000D1H   SFRSYM    DATA     BYTE      OADRL
      000000F0H.3 SFRSYM    DATA     BIT       B3
      000000F0H.4 SFRSYM    DATA     BIT       B4
      000000D0H.5 SFRSYM    DATA     BIT       F0
      000000F0H.5 SFRSYM    DATA     BIT       B5
      000000D0H.1 SFRSYM    DATA     BIT       F1
      000000AFH   SFRSYM    DATA     BYTE      REMAP
      000000F0H.6 SFRSYM    DATA     BIT       B6
      000000E0H.0 SFRSYM    DATA     BIT       ACC0
      000000A1H   SFRSYM    DATA     BYTE      OUS
      000000C8H.6 SFRSYM    DATA     BIT       PWM0S
      000000F0H.7 SFRSYM    DATA     BIT       B7
      000000E0H.1 SFRSYM    DATA     BIT       ACC1
      000000F8H.4 SFRSYM    DATA     BIT       XCLKF
      000000E0H.2 SFRSYM    DATA     BIT       ACC2
      0000008EH   SFRSYM    DATA     BYTE      PDSEL
      000000E0H.3 SFRSYM    DATA     BIT       ACC3
      000000D0H   SFRSYM    DATA     BYTE      PSW
      000000E0H.4 SFRSYM    DATA     BIT       ACC4
      00000098H.2 SFRSYM    DATA     BIT       RB80
      000000E0H.5 SFRSYM    DATA     BIT       ACC5
      000000FDH   SFRSYM    DATA     BYTE      ADCVREF
      000000E0H.6 SFRSYM    DATA     BIT       ACC6

      01000F65H   BLOCK     CODE     ---       LVL=0
      02000099H   SYMBOL    PDATA    DWORD     system_clk_hz
      01000F65H   LINE      CODE     ---       #22
      01000F6AH   LINE      CODE     ---       #23
      01000F6AH   LINE      CODE     ---       #24
      01000F6DH   LINE      CODE     ---       #25
      01000F75H   LINE      CODE     ---       #27
      01000F78H   LINE      CODE     ---       #28
      01000F7BH   LINE      CODE     ---       #30
      01000F7EH   LINE      CODE     ---       #31
      01000F81H   LINE      CODE     ---       #33
      ---         BLOCKEND  ---      ---       LVL=0

      01000026H   BLOCK     CODE     ---       LVL=0
      01000026H   LINE      CODE     ---       #42
      01000026H   LINE      CODE     ---       #43
      01000026H   LINE      CODE     ---       #44
      ---         BLOCKEND  ---      ---       LVL=0

      ---         MODULE    ---      ---       COMMON
      01000EFBH   PUBLIC    CODE     ---       _delay1ms
LX51 LINKER/LOCATER V4.66.97.0                                                        03/02/2021  17:27:53  PAGE 14


      00000098H.3 SFRSYM    DATA     BIT       TB80
      000000EDH   SFRSYM    DATA     BYTE      ADCCONT
      000000E0H.7 SFRSYM    DATA     BIT       ACC7
      00000080H   SFRSYM    DATA     BYTE      P0
      00000090H   SFRSYM    DATA     BYTE      P1
      000000A0H   SFRSYM    DATA     BYTE      P2
      00000098H.5 SFRSYM    DATA     BIT       SM20
      000000B2H   SFRSYM    DATA     BYTE      ESTCR
      000000B1H   SFRSYM    DATA     BYTE      CLKST
      000000D0H.6 SFRSYM    DATA     BIT       AC
      00000094H   SFRSYM    DATA     BYTE      PAGESEL
      000000D8H.3 SFRSYM    DATA     BIT       ERSTF
      000000E6H   SFRSYM    DATA     BYTE      PRESET0
      000000D4H   SFRSYM    DATA     BYTE      OCTRL
      000000A8H.7 SFRSYM    DATA     BIT       EA
      0000008FH   SFRSYM    DATA     BYTE      POREN
      000000C8H   SFRSYM    DATA     BYTE      PWM0CON
      000000E7H   SFRSYM    DATA     BYTE      PRESET1
      000000C9H   SFRSYM    DATA     BYTE      PWM1CON
      00000086H   SFRSYM    DATA     BYTE      BEEPCTR
      000000CAH   SFRSYM    DATA     BYTE      PWM2CON
      000000F8H.6 SFRSYM    DATA     BIT       RC32KF
      000000A8H   SFRSYM    DATA     BYTE      IEN0
      000000A7H   SFRSYM    DATA     BYTE      OPSET
      000000B8H   SFRSYM    DATA     BYTE      IEN1
      000000A8H.6 SFRSYM    DATA     BIT       EADC
      00000085H   SFRSYM    DATA     BYTE      DPH1
      000000B6H   SFRSYM    DATA     BYTE      ADCDR0
      000000F8H.5 SFRSYM    DATA     BIT       RC16MF
      000000B7H   SFRSYM    DATA     BYTE      ADCDR1
      00000084H   SFRSYM    DATA     BYTE      DPL1
      000000D6H   SFRSYM    DATA     BYTE      P0OD
      000000DBH   SFRSYM    DATA     BYTE      P1OD
      000000D5H   SFRSYM    DATA     BYTE      P0PD
      00000098H.4 SFRSYM    DATA     BIT       REN0
      000000ECH   SFRSYM    DATA     BYTE      P2OD
      000000DAH   SFRSYM    DATA     BYTE      P1PD
      000000E4H   SFRSYM    DATA     BYTE      P2PD
      000000D7H   SFRSYM    DATA     BYTE      P0CS
      00000097H   SFRSYM    DATA     BYTE      P0DR
      0000009EH   SFRSYM    DATA     BYTE      EUARTEN
      000000DCH   SFRSYM    DATA     BYTE      P1CS
      000000E5H   SFRSYM    DATA     BYTE      P1DR
      000000F4H   SFRSYM    DATA     BYTE      P2CS
      000000FCH   SFRSYM    DATA     BYTE      P2DR
      000000D0H.7 SFRSYM    DATA     BIT       CY
      000000D8H.0 SFRSYM    DATA     BIT       WDT0
      0000009FH   SFRSYM    DATA     BYTE      RCLTRIM
      000000D8H.1 SFRSYM    DATA     BIT       WDT1
      000000D8H.2 SFRSYM    DATA     BIT       WDT2
      00000081H   SFRSYM    DATA     BYTE      SP
      000000F1H   SFRSYM    DATA     BYTE      P0PU
      000000F2H   SFRSYM    DATA     BYTE      P1PU
      000000D1H   SFRSYM    DATA     WORD      OADR
      000000F3H   SFRSYM    DATA     BYTE      P2PU
      00000095H   SFRSYM    DATA     BYTE      D_PAGESEL
      00000093H   SFRSYM    DATA     BYTE      ADCIER
      000000D8H.6 SFRSYM    DATA     BIT       WDEN
      000000BAH   SFRSYM    DATA     BYTE      S0RELH
      00000080H.0 SFRSYM    DATA     BIT       P00
      000000D8H.7 SFRSYM    DATA     BIT       WDOF
      000000BBH   SFRSYM    DATA     BYTE      S1RELH
      00000090H.0 SFRSYM    DATA     BIT       P10
      00000080H.1 SFRSYM    DATA     BIT       P01
      00000087H   SFRSYM    DATA     BYTE      PCON
LX51 LINKER/LOCATER V4.66.97.0                                                        03/02/2021  17:27:53  PAGE 15


      000000C4H   SFRSYM    DATA     BYTE      PWM0DH
      000000A0H.0 SFRSYM    DATA     BIT       P20
      00000090H.1 SFRSYM    DATA     BIT       P11
      00000080H.2 SFRSYM    DATA     BIT       P02
      00000088H.0 SFRSYM    DATA     BIT       T0CLKS
      000000C6H   SFRSYM    DATA     BYTE      PWM1DH
      00000090H.2 SFRSYM    DATA     BIT       P12
      00000080H.3 SFRSYM    DATA     BIT       P03
      00000088H.4 SFRSYM    DATA     BIT       T1CLKS
      000000C7H   SFRSYM    DATA     BYTE      PWM2DH
      000000C8H.2 SFRSYM    DATA     BIT       PWM0IE
      000000AAH   SFRSYM    DATA     BYTE      S0RELL
      000000A0H.2 SFRSYM    DATA     BIT       P22
      00000090H.3 SFRSYM    DATA     BIT       P13
      00000080H.4 SFRSYM    DATA     BIT       P04
      00000089H   SFRSYM    DATA     BYTE      TMOD
      00000088H   SFRSYM    DATA     BYTE      TCON
      000000C8H.1 SFRSYM    DATA     BIT       PWM0IF
      0000009DH   SFRSYM    DATA     BYTE      S1RELL
      000000A0H.3 SFRSYM    DATA     BIT       P23
      00000090H.4 SFRSYM    DATA     BIT       P14
      000000C3H   SFRSYM    DATA     BYTE      PWM0DL
      00000090H.5 SFRSYM    DATA     BIT       P15
      000000A6H   SFRSYM    DATA     BYTE      OSTATUS
      000000C5H   SFRSYM    DATA     BYTE      PWM1DL
      000000A0H.5 SFRSYM    DATA     BIT       P25
      000000D8H.4 SFRSYM    DATA     BIT       PORF
      000000D8H   SFRSYM    DATA     BYTE      RSTSTAT
      000000CFH   SFRSYM    DATA     BYTE      PWM2DL
      000000A0H.6 SFRSYM    DATA     BIT       P26
      000000C8H.7 SFRSYM    DATA     BIT       PWM0EN
      000000A0H.7 SFRSYM    DATA     BIT       P27
      000000A8H.5 SFRSYM    DATA     BIT       EPWM
      000000D8H.5 SFRSYM    DATA     BIT       LVRF
      000000F8H   SFRSYM    DATA     BYTE      CLKCON
      000000CCH   SFRSYM    DATA     BYTE      PWM0PH
      000000CEH   SFRSYM    DATA     BYTE      PWM1PH
      000000C2H   SFRSYM    DATA     BYTE      PWM2PH
      000000F0H   SFRSYM    DATA     BYTE      B
      000000EEH   SFRSYM    DATA     BYTE      RCHDIV
      000000CBH   SFRSYM    DATA     BYTE      PWM0PL
      000000CDH   SFRSYM    DATA     BYTE      PWM1PL
      000000C1H   SFRSYM    DATA     BYTE      PWM2PL
      000000F7H   SFRSYM    DATA     BYTE      ADCSPW
      000000F8H.1 SFRSYM    DATA     BIT       XCLKEN
      000000E0H   SFRSYM    DATA     BYTE      ACC
      000000DDH   SFRSYM    DATA     BYTE      LVDCON
      000000A8H.4 SFRSYM    DATA     BIT       ES0
      000000A9H   SFRSYM    DATA     BYTE      IP0
      000000A8H.1 SFRSYM    DATA     BIT       ET0
      000000A8H.2 SFRSYM    DATA     BIT       ES1
      00000088H.3 SFRSYM    DATA     BIT       TF0
      000000F6H   SFRSYM    DATA     BYTE      ADCCSTAT
      000000B9H   SFRSYM    DATA     BYTE      IP1
      000000A8H.3 SFRSYM    DATA     BIT       ET1
      00000088H.7 SFRSYM    DATA     BIT       TF1
      00000098H.0 SFRSYM    DATA     BIT       RI0
      0000008CH   SFRSYM    DATA     BYTE      TH0
      000000C8H.0 SFRSYM    DATA     BIT       PWM0SS
      0000008DH   SFRSYM    DATA     BYTE      TH1
      00000098H.1 SFRSYM    DATA     BIT       TI0
      000000A8H.0 SFRSYM    DATA     BIT       EX0
      000000D0H.0 SFRSYM    DATA     BIT       P
      000000B8H.3 SFRSYM    DATA     BIT       EFCINTEN
      000000A2H   SFRSYM    DATA     BYTE      OINTEN
LX51 LINKER/LOCATER V4.66.97.0                                                        03/02/2021  17:27:53  PAGE 16


      0000008AH   SFRSYM    DATA     BYTE      TL0
      00000098H.7 SFRSYM    DATA     BIT       SM0
      0000008BH   SFRSYM    DATA     BYTE      TL1
      00000098H.6 SFRSYM    DATA     BIT       SM1
      000000FEH   SFRSYM    DATA     BYTE      ADCCDR0
      000000FFH   SFRSYM    DATA     BYTE      ADCCDR1
      000000D0H.3 SFRSYM    DATA     BIT       RS0
      00000088H.1 SFRSYM    DATA     BIT       TR0
      000000ACH   SFRSYM    DATA     BYTE      ADCGCR0
      000000D0H.4 SFRSYM    DATA     BIT       RS1
      00000088H.5 SFRSYM    DATA     BIT       TR1
      000000ADH   SFRSYM    DATA     BYTE      ADCGCR1
      000000B4H   SFRSYM    DATA     BYTE      ADCGCR2
      000000B5H   SFRSYM    DATA     BYTE      ADCGCR3
      000000F8H.3 SFRSYM    DATA     BIT       RC32KEN
      000000DEH   SFRSYM    DATA     BYTE      PCLK0
      000000DFH   SFRSYM    DATA     BYTE      PCLK1
      00000083H   SFRSYM    DATA     BYTE      DPH
      000000E9H   SFRSYM    DATA     BYTE      P0IEN
      000000F5H   SFRSYM    DATA     BYTE      ADCHL
      000000F8H.2 SFRSYM    DATA     BIT       RC16MEN
      000000EAH   SFRSYM    DATA     BYTE      P1IEN
      000000EBH   SFRSYM    DATA     BYTE      P2IEN
      000000B6H   SFRSYM    DATA     WORD      ADCDR
      000000B3H   SFRSYM    DATA     BYTE      XTHCTR
      00000082H   SFRSYM    DATA     BYTE      DPL
      00000099H   SFRSYM    DATA     BYTE      S0BUF
      0000009CH   SFRSYM    DATA     BYTE      S1BUF
      000000F9H   SFRSYM    DATA     BYTE      P0OEN
      000000D9H   SFRSYM    DATA     BYTE      SYSDIV
      00000098H   SFRSYM    DATA     BYTE      S0CON
      000000FAH   SFRSYM    DATA     BYTE      P1OEN
      000000A3H   SFRSYM    DATA     BYTE      OINTUS
      000000BEH   SFRSYM    DATA     BYTE      RCHTRIMH
      000000F8H.0 SFRSYM    DATA     BIT       SYSSEL
      0000009BH   SFRSYM    DATA     BYTE      S1CON
      000000FBH   SFRSYM    DATA     BYTE      P2OEN
      000000BDH   SFRSYM    DATA     BYTE      LDOTRIMH
      000000ABH   SFRSYM    DATA     BYTE      T2CON
      00000092H   SFRSYM    DATA     BYTE      DPS
      000000BFH   SFRSYM    DATA     BYTE      RCHTRIML
      000000D3H   SFRSYM    DATA     BYTE      ODATA
      00000091H   SFRSYM    DATA     BYTE      LDOTRIML
      000000E1H   SFRSYM    DATA     BYTE      P0IRQ
      000000B8H.1 SFRSYM    DATA     BIT       SPIINTEN
      000000E2H   SFRSYM    DATA     BYTE      P1IRQ
      000000E3H   SFRSYM    DATA     BYTE      P2IRQ
      000000D2H   SFRSYM    DATA     BYTE      OADRH
      000000F0H.0 SFRSYM    DATA     BIT       B0
      000000F0H.1 SFRSYM    DATA     BIT       B1
      000000F0H.2 SFRSYM    DATA     BIT       B2
      000000D1H   SFRSYM    DATA     BYTE      OADRL
      000000F0H.3 SFRSYM    DATA     BIT       B3
      000000F0H.4 SFRSYM    DATA     BIT       B4
      000000D0H.5 SFRSYM    DATA     BIT       F0
      000000F0H.5 SFRSYM    DATA     BIT       B5
      000000D0H.1 SFRSYM    DATA     BIT       F1
      000000AFH   SFRSYM    DATA     BYTE      REMAP
      000000F0H.6 SFRSYM    DATA     BIT       B6
      000000E0H.0 SFRSYM    DATA     BIT       ACC0
      000000A1H   SFRSYM    DATA     BYTE      OUS
      000000C8H.6 SFRSYM    DATA     BIT       PWM0S
      000000F0H.7 SFRSYM    DATA     BIT       B7
      000000E0H.1 SFRSYM    DATA     BIT       ACC1
      000000F8H.4 SFRSYM    DATA     BIT       XCLKF
LX51 LINKER/LOCATER V4.66.97.0                                                        03/02/2021  17:27:53  PAGE 17


      000000E0H.2 SFRSYM    DATA     BIT       ACC2
      0000008EH   SFRSYM    DATA     BYTE      PDSEL
      000000E0H.3 SFRSYM    DATA     BIT       ACC3
      000000D0H   SFRSYM    DATA     BYTE      PSW
      000000E0H.4 SFRSYM    DATA     BIT       ACC4
      00000098H.2 SFRSYM    DATA     BIT       RB80
      000000E0H.5 SFRSYM    DATA     BIT       ACC5
      000000FDH   SFRSYM    DATA     BYTE      ADCVREF
      000000E0H.6 SFRSYM    DATA     BIT       ACC6

      01000EFBH   BLOCK     CODE     ---       LVL=0
      0200009CH   SYMBOL    PDATA    DWORD     n
      01000F00H   BLOCK     CODE     NEAR LAB  LVL=1
      020000A0H   SYMBOL    PDATA    DWORD     x
      00000007H   SYMBOL    DATA     BYTE      i
      00000006H   SYMBOL    DATA     BYTE      j
      ---         BLOCKEND  ---      ---       LVL=1
      01000EFBH   LINE      CODE     ---       #21
      01000F00H   LINE      CODE     ---       #22
      01000F00H   LINE      CODE     ---       #26
      01000F19H   LINE      CODE     ---       #27
      01000F19H   LINE      CODE     ---       #28
      01000F1AH   LINE      CODE     ---       #29
      01000F1CH   LINE      CODE     ---       #30
      01000F1EH   LINE      CODE     ---       #32
      01000F1EH   LINE      CODE     ---       #33
      01000F20H   LINE      CODE     ---       #34
      01000F22H   LINE      CODE     ---       #35
      01000F3BH   LINE      CODE     ---       #36
      ---         BLOCKEND  ---      ---       LVL=0

      ---         MODULE    ---      ---       UART0
      020000B9H   PUBLIC    PDATA    BYTE      tx_flag
      020000B3H   PUBLIC    PDATA    ---       uart0func
      01001039H   PUBLIC    CODE     ---       _putchar
      0100103EH   PUBLIC    CODE     ---       uart0_recv_byte
      01000FC9H   PUBLIC    CODE     ---       _uart0_send_byte
      02000099H   PUBLIC    PDATA    BYTE      ?_uart0_irq_init?BYTE
      01000FACH   PUBLIC    CODE     ---       _uart0_irq_init
      01000EB9H   PUBLIC    CODE     ---       _uart0_init
      01000DFEH   PUBLIC    CODE     ---       UART0_IRQHandler
      00000098H.3 SFRSYM    DATA     BIT       TB80
      000000EDH   SFRSYM    DATA     BYTE      ADCCONT
      000000E0H.7 SFRSYM    DATA     BIT       ACC7
      00000080H   SFRSYM    DATA     BYTE      P0
      00000090H   SFRSYM    DATA     BYTE      P1
      000000A0H   SFRSYM    DATA     BYTE      P2
      00000098H.5 SFRSYM    DATA     BIT       SM20
      000000B2H   SFRSYM    DATA     BYTE      ESTCR
      000000B1H   SFRSYM    DATA     BYTE      CLKST
      000000D0H.6 SFRSYM    DATA     BIT       AC
      00000094H   SFRSYM    DATA     BYTE      PAGESEL
      000000D8H.3 SFRSYM    DATA     BIT       ERSTF
      000000E6H   SFRSYM    DATA     BYTE      PRESET0
      000000D4H   SFRSYM    DATA     BYTE      OCTRL
      000000A8H.7 SFRSYM    DATA     BIT       EA
      0000008FH   SFRSYM    DATA     BYTE      POREN
      000000C8H   SFRSYM    DATA     BYTE      PWM0CON
      000000E7H   SFRSYM    DATA     BYTE      PRESET1
      000000C9H   SFRSYM    DATA     BYTE      PWM1CON
      00000086H   SFRSYM    DATA     BYTE      BEEPCTR
      000000CAH   SFRSYM    DATA     BYTE      PWM2CON
      000000F8H.6 SFRSYM    DATA     BIT       RC32KF
      000000A8H   SFRSYM    DATA     BYTE      IEN0
      000000A7H   SFRSYM    DATA     BYTE      OPSET
LX51 LINKER/LOCATER V4.66.97.0                                                        03/02/2021  17:27:53  PAGE 18


      000000B8H   SFRSYM    DATA     BYTE      IEN1
      000000A8H.6 SFRSYM    DATA     BIT       EADC
      00000085H   SFRSYM    DATA     BYTE      DPH1
      000000B6H   SFRSYM    DATA     BYTE      ADCDR0
      000000F8H.5 SFRSYM    DATA     BIT       RC16MF
      000000B7H   SFRSYM    DATA     BYTE      ADCDR1
      00000084H   SFRSYM    DATA     BYTE      DPL1
      000000D6H   SFRSYM    DATA     BYTE      P0OD
      000000DBH   SFRSYM    DATA     BYTE      P1OD
      000000D5H   SFRSYM    DATA     BYTE      P0PD
      00000098H.4 SFRSYM    DATA     BIT       REN0
      000000ECH   SFRSYM    DATA     BYTE      P2OD
      000000DAH   SFRSYM    DATA     BYTE      P1PD
      000000E4H   SFRSYM    DATA     BYTE      P2PD
      000000D7H   SFRSYM    DATA     BYTE      P0CS
      00000097H   SFRSYM    DATA     BYTE      P0DR
      0000009EH   SFRSYM    DATA     BYTE      EUARTEN
      000000DCH   SFRSYM    DATA     BYTE      P1CS
      000000E5H   SFRSYM    DATA     BYTE      P1DR
      000000F4H   SFRSYM    DATA     BYTE      P2CS
      000000FCH   SFRSYM    DATA     BYTE      P2DR
      000000D0H.7 SFRSYM    DATA     BIT       CY
      000000D8H.0 SFRSYM    DATA     BIT       WDT0
      0000009FH   SFRSYM    DATA     BYTE      RCLTRIM
      000000D8H.1 SFRSYM    DATA     BIT       WDT1
      000000D8H.2 SFRSYM    DATA     BIT       WDT2
      00000081H   SFRSYM    DATA     BYTE      SP
      000000F1H   SFRSYM    DATA     BYTE      P0PU
      000000F2H   SFRSYM    DATA     BYTE      P1PU
      000000D1H   SFRSYM    DATA     WORD      OADR
      000000F3H   SFRSYM    DATA     BYTE      P2PU
      00000095H   SFRSYM    DATA     BYTE      D_PAGESEL
      00000093H   SFRSYM    DATA     BYTE      ADCIER
      000000D8H.6 SFRSYM    DATA     BIT       WDEN
      000000BAH   SFRSYM    DATA     BYTE      S0RELH
      00000080H.0 SFRSYM    DATA     BIT       P00
      000000D8H.7 SFRSYM    DATA     BIT       WDOF
      000000BBH   SFRSYM    DATA     BYTE      S1RELH
      00000090H.0 SFRSYM    DATA     BIT       P10
      00000080H.1 SFRSYM    DATA     BIT       P01
      00000087H   SFRSYM    DATA     BYTE      PCON
      000000C4H   SFRSYM    DATA     BYTE      PWM0DH
      000000A0H.0 SFRSYM    DATA     BIT       P20
      00000090H.1 SFRSYM    DATA     BIT       P11
      00000080H.2 SFRSYM    DATA     BIT       P02
      00000088H.0 SFRSYM    DATA     BIT       T0CLKS
      000000C6H   SFRSYM    DATA     BYTE      PWM1DH
      00000090H.2 SFRSYM    DATA     BIT       P12
      00000080H.3 SFRSYM    DATA     BIT       P03
      00000088H.4 SFRSYM    DATA     BIT       T1CLKS
      000000C7H   SFRSYM    DATA     BYTE      PWM2DH
      000000C8H.2 SFRSYM    DATA     BIT       PWM0IE
      000000AAH   SFRSYM    DATA     BYTE      S0RELL
      000000A0H.2 SFRSYM    DATA     BIT       P22
      00000090H.3 SFRSYM    DATA     BIT       P13
      00000080H.4 SFRSYM    DATA     BIT       P04
      00000089H   SFRSYM    DATA     BYTE      TMOD
      00000088H   SFRSYM    DATA     BYTE      TCON
      000000C8H.1 SFRSYM    DATA     BIT       PWM0IF
      0000009DH   SFRSYM    DATA     BYTE      S1RELL
      000000A0H.3 SFRSYM    DATA     BIT       P23
      00000090H.4 SFRSYM    DATA     BIT       P14
      000000C3H   SFRSYM    DATA     BYTE      PWM0DL
      00000090H.5 SFRSYM    DATA     BIT       P15
      000000A6H   SFRSYM    DATA     BYTE      OSTATUS
LX51 LINKER/LOCATER V4.66.97.0                                                        03/02/2021  17:27:53  PAGE 19


      000000C5H   SFRSYM    DATA     BYTE      PWM1DL
      000000A0H.5 SFRSYM    DATA     BIT       P25
      000000D8H.4 SFRSYM    DATA     BIT       PORF
      000000D8H   SFRSYM    DATA     BYTE      RSTSTAT
      000000CFH   SFRSYM    DATA     BYTE      PWM2DL
      000000A0H.6 SFRSYM    DATA     BIT       P26
      000000C8H.7 SFRSYM    DATA     BIT       PWM0EN
      000000A0H.7 SFRSYM    DATA     BIT       P27
      000000A8H.5 SFRSYM    DATA     BIT       EPWM
      000000D8H.5 SFRSYM    DATA     BIT       LVRF
      000000F8H   SFRSYM    DATA     BYTE      CLKCON
      000000CCH   SFRSYM    DATA     BYTE      PWM0PH
      000000CEH   SFRSYM    DATA     BYTE      PWM1PH
      000000C2H   SFRSYM    DATA     BYTE      PWM2PH
      000000F0H   SFRSYM    DATA     BYTE      B
      000000EEH   SFRSYM    DATA     BYTE      RCHDIV
      000000CBH   SFRSYM    DATA     BYTE      PWM0PL
      000000CDH   SFRSYM    DATA     BYTE      PWM1PL
      000000C1H   SFRSYM    DATA     BYTE      PWM2PL
      000000F7H   SFRSYM    DATA     BYTE      ADCSPW
      000000F8H.1 SFRSYM    DATA     BIT       XCLKEN
      000000E0H   SFRSYM    DATA     BYTE      ACC
      000000DDH   SFRSYM    DATA     BYTE      LVDCON
      000000A8H.4 SFRSYM    DATA     BIT       ES0
      000000A9H   SFRSYM    DATA     BYTE      IP0
      000000A8H.1 SFRSYM    DATA     BIT       ET0
      000000A8H.2 SFRSYM    DATA     BIT       ES1
      00000088H.3 SFRSYM    DATA     BIT       TF0
      000000F6H   SFRSYM    DATA     BYTE      ADCCSTAT
      000000B9H   SFRSYM    DATA     BYTE      IP1
      000000A8H.3 SFRSYM    DATA     BIT       ET1
      00000088H.7 SFRSYM    DATA     BIT       TF1
      00000098H.0 SFRSYM    DATA     BIT       RI0
      0000008CH   SFRSYM    DATA     BYTE      TH0
      000000C8H.0 SFRSYM    DATA     BIT       PWM0SS
      0000008DH   SFRSYM    DATA     BYTE      TH1
      00000098H.1 SFRSYM    DATA     BIT       TI0
      000000A8H.0 SFRSYM    DATA     BIT       EX0
      000000D0H.0 SFRSYM    DATA     BIT       P
      000000B8H.3 SFRSYM    DATA     BIT       EFCINTEN
      000000A2H   SFRSYM    DATA     BYTE      OINTEN
      0000008AH   SFRSYM    DATA     BYTE      TL0
      00000098H.7 SFRSYM    DATA     BIT       SM0
      0000008BH   SFRSYM    DATA     BYTE      TL1
      00000098H.6 SFRSYM    DATA     BIT       SM1
      000000FEH   SFRSYM    DATA     BYTE      ADCCDR0
      000000FFH   SFRSYM    DATA     BYTE      ADCCDR1
      000000D0H.3 SFRSYM    DATA     BIT       RS0
      00000088H.1 SFRSYM    DATA     BIT       TR0
      000000ACH   SFRSYM    DATA     BYTE      ADCGCR0
      000000D0H.4 SFRSYM    DATA     BIT       RS1
      00000088H.5 SFRSYM    DATA     BIT       TR1
      000000ADH   SFRSYM    DATA     BYTE      ADCGCR1
      000000B4H   SFRSYM    DATA     BYTE      ADCGCR2
      000000B5H   SFRSYM    DATA     BYTE      ADCGCR3
      000000F8H.3 SFRSYM    DATA     BIT       RC32KEN
      000000DEH   SFRSYM    DATA     BYTE      PCLK0
      000000DFH   SFRSYM    DATA     BYTE      PCLK1
      00000083H   SFRSYM    DATA     BYTE      DPH
      000000E9H   SFRSYM    DATA     BYTE      P0IEN
      000000F5H   SFRSYM    DATA     BYTE      ADCHL
      000000F8H.2 SFRSYM    DATA     BIT       RC16MEN
      000000EAH   SFRSYM    DATA     BYTE      P1IEN
      000000EBH   SFRSYM    DATA     BYTE      P2IEN
      000000B6H   SFRSYM    DATA     WORD      ADCDR
LX51 LINKER/LOCATER V4.66.97.0                                                        03/02/2021  17:27:53  PAGE 20


      000000B3H   SFRSYM    DATA     BYTE      XTHCTR
      00000082H   SFRSYM    DATA     BYTE      DPL
      00000099H   SFRSYM    DATA     BYTE      S0BUF
      0000009CH   SFRSYM    DATA     BYTE      S1BUF
      000000F9H   SFRSYM    DATA     BYTE      P0OEN
      000000D9H   SFRSYM    DATA     BYTE      SYSDIV
      00000098H   SFRSYM    DATA     BYTE      S0CON
      000000FAH   SFRSYM    DATA     BYTE      P1OEN
      000000A3H   SFRSYM    DATA     BYTE      OINTUS
      000000BEH   SFRSYM    DATA     BYTE      RCHTRIMH
      000000F8H.0 SFRSYM    DATA     BIT       SYSSEL
      0000009BH   SFRSYM    DATA     BYTE      S1CON
      000000FBH   SFRSYM    DATA     BYTE      P2OEN
      000000BDH   SFRSYM    DATA     BYTE      LDOTRIMH
      000000ABH   SFRSYM    DATA     BYTE      T2CON
      00000092H   SFRSYM    DATA     BYTE      DPS
      000000BFH   SFRSYM    DATA     BYTE      RCHTRIML
      000000D3H   SFRSYM    DATA     BYTE      ODATA
      00000091H   SFRSYM    DATA     BYTE      LDOTRIML
      000000E1H   SFRSYM    DATA     BYTE      P0IRQ
      000000B8H.1 SFRSYM    DATA     BIT       SPIINTEN
      000000E2H   SFRSYM    DATA     BYTE      P1IRQ
      000000E3H   SFRSYM    DATA     BYTE      P2IRQ
      000000D2H   SFRSYM    DATA     BYTE      OADRH
      000000F0H.0 SFRSYM    DATA     BIT       B0
      000000F0H.1 SFRSYM    DATA     BIT       B1
      000000F0H.2 SFRSYM    DATA     BIT       B2
      000000D1H   SFRSYM    DATA     BYTE      OADRL
      000000F0H.3 SFRSYM    DATA     BIT       B3
      000000F0H.4 SFRSYM    DATA     BIT       B4
      000000D0H.5 SFRSYM    DATA     BIT       F0
      000000F0H.5 SFRSYM    DATA     BIT       B5
      000000D0H.1 SFRSYM    DATA     BIT       F1
      000000AFH   SFRSYM    DATA     BYTE      REMAP
      000000F0H.6 SFRSYM    DATA     BIT       B6
      000000E0H.0 SFRSYM    DATA     BIT       ACC0
      000000A1H   SFRSYM    DATA     BYTE      OUS
      000000C8H.6 SFRSYM    DATA     BIT       PWM0S
      000000F0H.7 SFRSYM    DATA     BIT       B7
      000000E0H.1 SFRSYM    DATA     BIT       ACC1
      000000F8H.4 SFRSYM    DATA     BIT       XCLKF
      000000E0H.2 SFRSYM    DATA     BIT       ACC2
      0000008EH   SFRSYM    DATA     BYTE      PDSEL
      000000E0H.3 SFRSYM    DATA     BIT       ACC3
      000000D0H   SFRSYM    DATA     BYTE      PSW
      000000E0H.4 SFRSYM    DATA     BIT       ACC4
      00000098H.2 SFRSYM    DATA     BIT       RB80
      000000E0H.5 SFRSYM    DATA     BIT       ACC5
      000000FDH   SFRSYM    DATA     BYTE      ADCVREF
      000000E0H.6 SFRSYM    DATA     BIT       ACC6
      01000D25H   SYMBOL    CODE     ---       _uart0_set_baud_rate

      01000DFEH   BLOCK     CODE     ---       LVL=0
      01000DFEH   LINE      CODE     ---       #24
      01000E25H   LINE      CODE     ---       #26
      01000E28H   LINE      CODE     ---       #27
      01000E28H   LINE      CODE     ---       #28
      01000E32H   LINE      CODE     ---       #29
      01000E32H   LINE      CODE     ---       #30
      01000E3AH   LINE      CODE     ---       #31
      01000E3AH   LINE      CODE     ---       #32
      01000E3CH   LINE      CODE     ---       #33
      01000E3CH   LINE      CODE     ---       #45
      ---         BLOCKEND  ---      ---       LVL=0

LX51 LINKER/LOCATER V4.66.97.0                                                        03/02/2021  17:27:53  PAGE 21


      01000D25H   BLOCK     CODE     ---       LVL=0
      0200009DH   SYMBOL    PDATA    DWORD     clk_hz
      020000A1H   SYMBOL    PDATA    DWORD     baud_rate
      01000D2AH   BLOCK     CODE     NEAR LAB  LVL=1
      020000A5H   SYMBOL    PDATA    DWORD     temp
      00000003H   SYMBOL    DATA     BYTE      MSbyte
      00000007H   SYMBOL    DATA     BYTE      LSbyte
      ---         BLOCKEND  ---      ---       LVL=1
      01000D25H   LINE      CODE     ---       #57
      01000D2AH   LINE      CODE     ---       #58
      01000D2AH   LINE      CODE     ---       #62
      01000D3DH   LINE      CODE     ---       #63
      01000D64H   LINE      CODE     ---       #64
      01000D7CH   LINE      CODE     ---       #66
      01000D88H   LINE      CODE     ---       #67
      01000D8DH   LINE      CODE     ---       #69
      01000D92H   LINE      CODE     ---       #70
      01000D94H   LINE      CODE     ---       #71
      ---         BLOCKEND  ---      ---       LVL=0

      01000EB9H   BLOCK     CODE     ---       LVL=0
      02000099H   SYMBOL    PDATA    DWORD     baud_rate
      01000EBEH   BLOCK     CODE     NEAR LAB  LVL=1
      00000004H   SYMBOL    DATA     DWORD     uart_clk_hz
      ---         BLOCKEND  ---      ---       LVL=1
      01000EB9H   LINE      CODE     ---       #81
      01000EBEH   LINE      CODE     ---       #82
      01000EBEH   LINE      CODE     ---       #84
      01000EC6H   LINE      CODE     ---       #86
      01000EC9H   LINE      CODE     ---       #87
      01000ECCH   LINE      CODE     ---       #88
      01000ECFH   LINE      CODE     ---       #90
      01000ED3H   LINE      CODE     ---       #92
      01000ED5H   LINE      CODE     ---       #93
      01000ED7H   LINE      CODE     ---       #95
      01000ED9H   LINE      CODE     ---       #96
      01000EDBH   LINE      CODE     ---       #98
      01000EF8H   LINE      CODE     ---       #99
      01000EFAH   LINE      CODE     ---       #101
      ---         BLOCKEND  ---      ---       LVL=0

      01000FACH   BLOCK     CODE     ---       LVL=0
      00000007H   SYMBOL    DATA     BYTE      irqstate
      00000001H   SYMBOL    DATA     ---       pfunc_rec
      0200009DH   SYMBOL    PDATA    ---       pfunc_send
      01000FACH   LINE      CODE     ---       #111
      01000FACH   LINE      CODE     ---       #112
      01000FACH   LINE      CODE     ---       #113
      01000FB1H   LINE      CODE     ---       #114
      01000FB1H   LINE      CODE     ---       #115
      01000FB3H   LINE      CODE     ---       #116
      01000FB5H   LINE      CODE     ---       #118
      01000FBAH   LINE      CODE     ---       #119
      01000FC4H   LINE      CODE     ---       #120
      01000FC4H   LINE      CODE     ---       #122
      01000FC4H   LINE      CODE     ---       #123
      01000FC6H   LINE      CODE     ---       #124
      01000FC8H   LINE      CODE     ---       #125
      01000FC8H   LINE      CODE     ---       #126
      ---         BLOCKEND  ---      ---       LVL=0

      01000FC9H   BLOCK     CODE     ---       LVL=0
      00000007H   SYMBOL    DATA     CHAR      c
      01000FC9H   BLOCK     CODE     NEAR LAB  LVL=1
      00000004H   SYMBOL    DATA     WORD      timeout
LX51 LINKER/LOCATER V4.66.97.0                                                        03/02/2021  17:27:53  PAGE 22


      ---         BLOCKEND  ---      ---       LVL=1
      01000FC9H   LINE      CODE     ---       #137
      01000FC9H   LINE      CODE     ---       #138
      01000FC9H   LINE      CODE     ---       #141
      01000FCDH   LINE      CODE     ---       #143
      01000FCFH   LINE      CODE     ---       #150
      01000FD2H   LINE      CODE     ---       #151
      01000FD2H   LINE      CODE     ---       #152
      01000FDCH   LINE      CODE     ---       #153
      01000FDCH   LINE      CODE     ---       #154
      01000FDCH   LINE      CODE     ---       #155
      01000FDCH   LINE      CODE     ---       #156
      01000FDCH   LINE      CODE     ---       #157
      01000FDEH   LINE      CODE     ---       #159
      ---         BLOCKEND  ---      ---       LVL=0

      0100103EH   BLOCK     CODE     ---       LVL=0
      0100103EH   BLOCK     CODE     NEAR LAB  LVL=1
      00000007H   SYMBOL    DATA     BYTE      recv_data
      ---         BLOCKEND  ---      ---       LVL=1
      0100103EH   LINE      CODE     ---       #184
      0100103EH   LINE      CODE     ---       #185
      0100103EH   LINE      CODE     ---       #186
      0100103EH   LINE      CODE     ---       #188
      01001040H   LINE      CODE     ---       #190
      01001040H   LINE      CODE     ---       #191
      ---         BLOCKEND  ---      ---       LVL=0

      01001039H   BLOCK     CODE     ---       LVL=0
      00000003H   SYMBOL    DATA     CHAR      c
      01001039H   LINE      CODE     ---       #200
      0100103BH   LINE      CODE     ---       #201
      0100103BH   LINE      CODE     ---       #202
      ---         BLOCKEND  ---      ---       LVL=0

      ---         MODULE    ---      ---       ADC
      020000BEH   PUBLIC    PDATA    ---       adcfunc
      01000FF5H   PUBLIC    CODE     ---       _get_adc
      0100102BH   PUBLIC    CODE     ---       get_adc_value
      01001012H   PUBLIC    CODE     ---       _adc_convert_start
      01001004H   PUBLIC    CODE     ---       _adc_io_config
      0200009CH   PUBLIC    PDATA    BYTE      ?_adc_init?BYTE
      01000E61H   PUBLIC    CODE     ---       _adc_init
      01000D95H   PUBLIC    CODE     ---       ADC_IRQHandler
      00000098H.3 SFRSYM    DATA     BIT       TB80
      000000EDH   SFRSYM    DATA     BYTE      ADCCONT
      000000E0H.7 SFRSYM    DATA     BIT       ACC7
      00000080H   SFRSYM    DATA     BYTE      P0
      00000090H   SFRSYM    DATA     BYTE      P1
      000000A0H   SFRSYM    DATA     BYTE      P2
      00000098H.5 SFRSYM    DATA     BIT       SM20
      000000B2H   SFRSYM    DATA     BYTE      ESTCR
      000000B1H   SFRSYM    DATA     BYTE      CLKST
      000000D0H.6 SFRSYM    DATA     BIT       AC
      00000094H   SFRSYM    DATA     BYTE      PAGESEL
      000000D8H.3 SFRSYM    DATA     BIT       ERSTF
      000000E6H   SFRSYM    DATA     BYTE      PRESET0
      000000D4H   SFRSYM    DATA     BYTE      OCTRL
      000000A8H.7 SFRSYM    DATA     BIT       EA
      0000008FH   SFRSYM    DATA     BYTE      POREN
      000000C8H   SFRSYM    DATA     BYTE      PWM0CON
      000000E7H   SFRSYM    DATA     BYTE      PRESET1
      000000C9H   SFRSYM    DATA     BYTE      PWM1CON
      00000086H   SFRSYM    DATA     BYTE      BEEPCTR
      000000CAH   SFRSYM    DATA     BYTE      PWM2CON
LX51 LINKER/LOCATER V4.66.97.0                                                        03/02/2021  17:27:53  PAGE 23


      000000F8H.6 SFRSYM    DATA     BIT       RC32KF
      000000A8H   SFRSYM    DATA     BYTE      IEN0
      000000A7H   SFRSYM    DATA     BYTE      OPSET
      000000B8H   SFRSYM    DATA     BYTE      IEN1
      000000A8H.6 SFRSYM    DATA     BIT       EADC
      00000085H   SFRSYM    DATA     BYTE      DPH1
      000000B6H   SFRSYM    DATA     BYTE      ADCDR0
      000000F8H.5 SFRSYM    DATA     BIT       RC16MF
      000000B7H   SFRSYM    DATA     BYTE      ADCDR1
      00000084H   SFRSYM    DATA     BYTE      DPL1
      000000D6H   SFRSYM    DATA     BYTE      P0OD
      000000DBH   SFRSYM    DATA     BYTE      P1OD
      000000D5H   SFRSYM    DATA     BYTE      P0PD
      00000098H.4 SFRSYM    DATA     BIT       REN0
      000000ECH   SFRSYM    DATA     BYTE      P2OD
      000000DAH   SFRSYM    DATA     BYTE      P1PD
      000000E4H   SFRSYM    DATA     BYTE      P2PD
      000000D7H   SFRSYM    DATA     BYTE      P0CS
      00000097H   SFRSYM    DATA     BYTE      P0DR
      0000009EH   SFRSYM    DATA     BYTE      EUARTEN
      000000DCH   SFRSYM    DATA     BYTE      P1CS
      000000E5H   SFRSYM    DATA     BYTE      P1DR
      000000F4H   SFRSYM    DATA     BYTE      P2CS
      000000FCH   SFRSYM    DATA     BYTE      P2DR
      000000D0H.7 SFRSYM    DATA     BIT       CY
      000000D8H.0 SFRSYM    DATA     BIT       WDT0
      0000009FH   SFRSYM    DATA     BYTE      RCLTRIM
      000000D8H.1 SFRSYM    DATA     BIT       WDT1
      000000D8H.2 SFRSYM    DATA     BIT       WDT2
      00000081H   SFRSYM    DATA     BYTE      SP
      000000F1H   SFRSYM    DATA     BYTE      P0PU
      000000F2H   SFRSYM    DATA     BYTE      P1PU
      000000D1H   SFRSYM    DATA     WORD      OADR
      000000F3H   SFRSYM    DATA     BYTE      P2PU
      00000095H   SFRSYM    DATA     BYTE      D_PAGESEL
      00000093H   SFRSYM    DATA     BYTE      ADCIER
      000000D8H.6 SFRSYM    DATA     BIT       WDEN
      000000BAH   SFRSYM    DATA     BYTE      S0RELH
      00000080H.0 SFRSYM    DATA     BIT       P00
      000000D8H.7 SFRSYM    DATA     BIT       WDOF
      000000BBH   SFRSYM    DATA     BYTE      S1RELH
      00000090H.0 SFRSYM    DATA     BIT       P10
      00000080H.1 SFRSYM    DATA     BIT       P01
      00000087H   SFRSYM    DATA     BYTE      PCON
      000000C4H   SFRSYM    DATA     BYTE      PWM0DH
      000000A0H.0 SFRSYM    DATA     BIT       P20
      00000090H.1 SFRSYM    DATA     BIT       P11
      00000080H.2 SFRSYM    DATA     BIT       P02
      00000088H.0 SFRSYM    DATA     BIT       T0CLKS
      000000C6H   SFRSYM    DATA     BYTE      PWM1DH
      00000090H.2 SFRSYM    DATA     BIT       P12
      00000080H.3 SFRSYM    DATA     BIT       P03
      00000088H.4 SFRSYM    DATA     BIT       T1CLKS
      000000C7H   SFRSYM    DATA     BYTE      PWM2DH
      000000C8H.2 SFRSYM    DATA     BIT       PWM0IE
      000000AAH   SFRSYM    DATA     BYTE      S0RELL
      000000A0H.2 SFRSYM    DATA     BIT       P22
      00000090H.3 SFRSYM    DATA     BIT       P13
      00000080H.4 SFRSYM    DATA     BIT       P04
      00000089H   SFRSYM    DATA     BYTE      TMOD
      00000088H   SFRSYM    DATA     BYTE      TCON
      000000C8H.1 SFRSYM    DATA     BIT       PWM0IF
      0000009DH   SFRSYM    DATA     BYTE      S1RELL
      000000A0H.3 SFRSYM    DATA     BIT       P23
      00000090H.4 SFRSYM    DATA     BIT       P14
LX51 LINKER/LOCATER V4.66.97.0                                                        03/02/2021  17:27:53  PAGE 24


      000000C3H   SFRSYM    DATA     BYTE      PWM0DL
      00000090H.5 SFRSYM    DATA     BIT       P15
      000000A6H   SFRSYM    DATA     BYTE      OSTATUS
      000000C5H   SFRSYM    DATA     BYTE      PWM1DL
      000000A0H.5 SFRSYM    DATA     BIT       P25
      000000D8H.4 SFRSYM    DATA     BIT       PORF
      000000D8H   SFRSYM    DATA     BYTE      RSTSTAT
      000000CFH   SFRSYM    DATA     BYTE      PWM2DL
      000000A0H.6 SFRSYM    DATA     BIT       P26
      000000C8H.7 SFRSYM    DATA     BIT       PWM0EN
      000000A0H.7 SFRSYM    DATA     BIT       P27
      000000A8H.5 SFRSYM    DATA     BIT       EPWM
      000000D8H.5 SFRSYM    DATA     BIT       LVRF
      000000F8H   SFRSYM    DATA     BYTE      CLKCON
      000000CCH   SFRSYM    DATA     BYTE      PWM0PH
      000000CEH   SFRSYM    DATA     BYTE      PWM1PH
      000000C2H   SFRSYM    DATA     BYTE      PWM2PH
      000000F0H   SFRSYM    DATA     BYTE      B
      000000EEH   SFRSYM    DATA     BYTE      RCHDIV
      000000CBH   SFRSYM    DATA     BYTE      PWM0PL
      000000CDH   SFRSYM    DATA     BYTE      PWM1PL
      000000C1H   SFRSYM    DATA     BYTE      PWM2PL
      000000F7H   SFRSYM    DATA     BYTE      ADCSPW
      000000F8H.1 SFRSYM    DATA     BIT       XCLKEN
      000000E0H   SFRSYM    DATA     BYTE      ACC
      000000DDH   SFRSYM    DATA     BYTE      LVDCON
      000000A8H.4 SFRSYM    DATA     BIT       ES0
      000000A9H   SFRSYM    DATA     BYTE      IP0
      000000A8H.1 SFRSYM    DATA     BIT       ET0
      000000A8H.2 SFRSYM    DATA     BIT       ES1
      00000088H.3 SFRSYM    DATA     BIT       TF0
      000000F6H   SFRSYM    DATA     BYTE      ADCCSTAT
      000000B9H   SFRSYM    DATA     BYTE      IP1
      000000A8H.3 SFRSYM    DATA     BIT       ET1
      00000088H.7 SFRSYM    DATA     BIT       TF1
      00000098H.0 SFRSYM    DATA     BIT       RI0
      0000008CH   SFRSYM    DATA     BYTE      TH0
      000000C8H.0 SFRSYM    DATA     BIT       PWM0SS
      0000008DH   SFRSYM    DATA     BYTE      TH1
      00000098H.1 SFRSYM    DATA     BIT       TI0
      000000A8H.0 SFRSYM    DATA     BIT       EX0
      000000D0H.0 SFRSYM    DATA     BIT       P
      000000B8H.3 SFRSYM    DATA     BIT       EFCINTEN
      000000A2H   SFRSYM    DATA     BYTE      OINTEN
      0000008AH   SFRSYM    DATA     BYTE      TL0
      00000098H.7 SFRSYM    DATA     BIT       SM0
      0000008BH   SFRSYM    DATA     BYTE      TL1
      00000098H.6 SFRSYM    DATA     BIT       SM1
      000000FEH   SFRSYM    DATA     BYTE      ADCCDR0
      000000FFH   SFRSYM    DATA     BYTE      ADCCDR1
      000000D0H.3 SFRSYM    DATA     BIT       RS0
      00000088H.1 SFRSYM    DATA     BIT       TR0
      000000ACH   SFRSYM    DATA     BYTE      ADCGCR0
      000000D0H.4 SFRSYM    DATA     BIT       RS1
      00000088H.5 SFRSYM    DATA     BIT       TR1
      000000ADH   SFRSYM    DATA     BYTE      ADCGCR1
      000000B4H   SFRSYM    DATA     BYTE      ADCGCR2
      000000B5H   SFRSYM    DATA     BYTE      ADCGCR3
      000000F8H.3 SFRSYM    DATA     BIT       RC32KEN
      000000DEH   SFRSYM    DATA     BYTE      PCLK0
      000000DFH   SFRSYM    DATA     BYTE      PCLK1
      00000083H   SFRSYM    DATA     BYTE      DPH
      000000E9H   SFRSYM    DATA     BYTE      P0IEN
      000000F5H   SFRSYM    DATA     BYTE      ADCHL
      000000F8H.2 SFRSYM    DATA     BIT       RC16MEN
LX51 LINKER/LOCATER V4.66.97.0                                                        03/02/2021  17:27:53  PAGE 25


      000000EAH   SFRSYM    DATA     BYTE      P1IEN
      000000EBH   SFRSYM    DATA     BYTE      P2IEN
      000000B6H   SFRSYM    DATA     WORD      ADCDR
      000000B3H   SFRSYM    DATA     BYTE      XTHCTR
      00000082H   SFRSYM    DATA     BYTE      DPL
      00000099H   SFRSYM    DATA     BYTE      S0BUF
      0000009CH   SFRSYM    DATA     BYTE      S1BUF
      000000F9H   SFRSYM    DATA     BYTE      P0OEN
      000000D9H   SFRSYM    DATA     BYTE      SYSDIV
      00000098H   SFRSYM    DATA     BYTE      S0CON
      000000FAH   SFRSYM    DATA     BYTE      P1OEN
      000000A3H   SFRSYM    DATA     BYTE      OINTUS
      000000BEH   SFRSYM    DATA     BYTE      RCHTRIMH
      000000F8H.0 SFRSYM    DATA     BIT       SYSSEL
      0000009BH   SFRSYM    DATA     BYTE      S1CON
      000000FBH   SFRSYM    DATA     BYTE      P2OEN
      000000BDH   SFRSYM    DATA     BYTE      LDOTRIMH
      000000ABH   SFRSYM    DATA     BYTE      T2CON
      00000092H   SFRSYM    DATA     BYTE      DPS
      000000BFH   SFRSYM    DATA     BYTE      RCHTRIML
      000000D3H   SFRSYM    DATA     BYTE      ODATA
      00000091H   SFRSYM    DATA     BYTE      LDOTRIML
      000000E1H   SFRSYM    DATA     BYTE      P0IRQ
      000000B8H.1 SFRSYM    DATA     BIT       SPIINTEN
      000000E2H   SFRSYM    DATA     BYTE      P1IRQ
      000000E3H   SFRSYM    DATA     BYTE      P2IRQ
      000000D2H   SFRSYM    DATA     BYTE      OADRH
      000000F0H.0 SFRSYM    DATA     BIT       B0
      000000F0H.1 SFRSYM    DATA     BIT       B1
      000000F0H.2 SFRSYM    DATA     BIT       B2
      000000D1H   SFRSYM    DATA     BYTE      OADRL
      000000F0H.3 SFRSYM    DATA     BIT       B3
      000000F0H.4 SFRSYM    DATA     BIT       B4
      000000D0H.5 SFRSYM    DATA     BIT       F0
      000000F0H.5 SFRSYM    DATA     BIT       B5
      000000D0H.1 SFRSYM    DATA     BIT       F1
      000000AFH   SFRSYM    DATA     BYTE      REMAP
      000000F0H.6 SFRSYM    DATA     BIT       B6
      000000E0H.0 SFRSYM    DATA     BIT       ACC0
      000000A1H   SFRSYM    DATA     BYTE      OUS
      000000C8H.6 SFRSYM    DATA     BIT       PWM0S
      000000F0H.7 SFRSYM    DATA     BIT       B7
      000000E0H.1 SFRSYM    DATA     BIT       ACC1
      000000F8H.4 SFRSYM    DATA     BIT       XCLKF
      000000E0H.2 SFRSYM    DATA     BIT       ACC2
      0000008EH   SFRSYM    DATA     BYTE      PDSEL
      000000E0H.3 SFRSYM    DATA     BIT       ACC3
      000000D0H   SFRSYM    DATA     BYTE      PSW
      000000E0H.4 SFRSYM    DATA     BIT       ACC4
      00000098H.2 SFRSYM    DATA     BIT       RB80
      000000E0H.5 SFRSYM    DATA     BIT       ACC5
      000000FDH   SFRSYM    DATA     BYTE      ADCVREF
      000000E0H.6 SFRSYM    DATA     BIT       ACC6

      01000D95H   BLOCK     CODE     ---       LVL=0
      01000D95H   LINE      CODE     ---       #21
      01000DBCH   LINE      CODE     ---       #24
      01000DC4H   LINE      CODE     ---       #25
      01000DC4H   LINE      CODE     ---       #26
      01000DCEH   LINE      CODE     ---       #27
      01000DCEH   LINE      CODE     ---       #28
      01000DD6H   LINE      CODE     ---       #29
      01000DD6H   LINE      CODE     ---       #30
      01000DD9H   LINE      CODE     ---       #31
      01000DD9H   LINE      CODE     ---       #33
LX51 LINKER/LOCATER V4.66.97.0                                                        03/02/2021  17:27:53  PAGE 26


      ---         BLOCKEND  ---      ---       LVL=0

      01000E61H   BLOCK     CODE     ---       LVL=0
      00000007H   SYMBOL    DATA     BYTE      adc_vref
      00000005H   SYMBOL    DATA     BYTE      adc_clk
      00000002H   SYMBOL    DATA     WORD      div
      020000A0H   SYMBOL    PDATA    BYTE      work_mode
      01000E61H   LINE      CODE     ---       #45
      01000E61H   LINE      CODE     ---       #46
      01000E61H   LINE      CODE     ---       #48
      01000E64H   LINE      CODE     ---       #49
      01000E67H   LINE      CODE     ---       #51
      01000E6AH   LINE      CODE     ---       #53
      01000E6DH   LINE      CODE     ---       #54
      01000E70H   LINE      CODE     ---       #56
      01000E73H   LINE      CODE     ---       #57
      01000E73H   LINE      CODE     ---       #58
      01000E76H   LINE      CODE     ---       #59
      01000E78H   LINE      CODE     ---       #61
      01000E78H   LINE      CODE     ---       #62
      01000E7BH   LINE      CODE     ---       #63
      01000E7BH   LINE      CODE     ---       #65
      01000E7EH   LINE      CODE     ---       #66
      01000E7EH   LINE      CODE     ---       #67
      01000E81H   LINE      CODE     ---       #68
      01000E83H   LINE      CODE     ---       #70
      01000E83H   LINE      CODE     ---       #71
      01000E86H   LINE      CODE     ---       #72
      01000E86H   LINE      CODE     ---       #74
      01000E8BH   LINE      CODE     ---       #75
      01000E8BH   LINE      CODE     ---       #76
      01000E8EH   LINE      CODE     ---       #77
      01000E90H   LINE      CODE     ---       #79
      01000E90H   LINE      CODE     ---       #80
      01000E93H   LINE      CODE     ---       #81
      01000E93H   LINE      CODE     ---       #83
      01000E96H   LINE      CODE     ---       #85
      01000E99H   LINE      CODE     ---       #89
      01000E9CH   LINE      CODE     ---       #90
      01000E9EH   LINE      CODE     ---       #91
      01000EA1H   LINE      CODE     ---       #92
      01000EA4H   LINE      CODE     ---       #94
      01000EA7H   LINE      CODE     ---       #97
      01000EAAH   LINE      CODE     ---       #98
      01000EADH   LINE      CODE     ---       #99
      01000EB2H   LINE      CODE     ---       #100
      01000EB5H   LINE      CODE     ---       #101
      01000EB8H   LINE      CODE     ---       #103
      ---         BLOCKEND  ---      ---       LVL=0

      01001004H   BLOCK     CODE     ---       LVL=0
      00000007H   SYMBOL    DATA     BYTE      ch
      01001004H   LINE      CODE     ---       #123
      01001004H   LINE      CODE     ---       #124
      01001004H   LINE      CODE     ---       #125
      01001011H   LINE      CODE     ---       #126
      ---         BLOCKEND  ---      ---       LVL=0
      00000007H   SYMBOL    DATA     BYTE      adc_irq_enable
      00000001H   SYMBOL    DATA     ---       pfunc

      01001012H   BLOCK     CODE     ---       LVL=0
      00000007H   SYMBOL    DATA     BYTE      ch
      01001012H   LINE      CODE     ---       #157
      01001012H   LINE      CODE     ---       #158
      01001012H   LINE      CODE     ---       #159
LX51 LINKER/LOCATER V4.66.97.0                                                        03/02/2021  17:27:53  PAGE 27


      01001015H   LINE      CODE     ---       #160
      01001019H   LINE      CODE     ---       #162
      0100101CH   LINE      CODE     ---       #163
      0100101FH   LINE      CODE     ---       #165
      ---         BLOCKEND  ---      ---       LVL=0

      0100102BH   BLOCK     CODE     ---       LVL=0
      0100102BH   LINE      CODE     ---       #185
      0100102BH   LINE      CODE     ---       #186
      0100102BH   LINE      CODE     ---       #187
      01001032H   LINE      CODE     ---       #189
      ---         BLOCKEND  ---      ---       LVL=0

      01000FF5H   BLOCK     CODE     ---       LVL=0
      00000007H   SYMBOL    DATA     BYTE      ch
      01000FF5H   BLOCK     CODE     NEAR LAB  LVL=1
      00000006H   SYMBOL    DATA     WORD      adc_value
      ---         BLOCKEND  ---      ---       LVL=1
      01000FF5H   LINE      CODE     ---       #197
      01000FF5H   LINE      CODE     ---       #198
      01000FF5H   LINE      CODE     ---       #201
      01000FF8H   LINE      CODE     ---       #203
      01000FFDH   LINE      CODE     ---       #204
      01001000H   LINE      CODE     ---       #206
      01001003H   LINE      CODE     ---       #208
      01001003H   LINE      CODE     ---       #210
      ---         BLOCKEND  ---      ---       LVL=0

      ---         MODULE    ---      ---       APP
      02000097H   PUBLIC    PDATA    WORD      tx_count
      02000095H   PUBLIC    PDATA    WORD      rx_count
      02000094H   PUBLIC    PDATA    BYTE      adc_rx_flag
      02000093H   PUBLIC    PDATA    BYTE      rx_flag
      02000073H   PUBLIC    PDATA    ---       uart0_tx_buf
      02000053H   PUBLIC    PDATA    ---       uart0_rx_buf
      02000051H   PUBLIC    PDATA    WORD      adc_data
      02000001H   PUBLIC    PDATA    ---       adc_converte_val
      02000000H   PUBLIC    PDATA    BYTE      adc_rx_count
      01000FDFH   PUBLIC    CODE     ---       adc_test
      01000CB0H   PUBLIC    CODE     ---       adc_single_mode_test
      01000F8BH   PUBLIC    CODE     ---       uart_init
      01001033H   PUBLIC    CODE     ---       uart0_send_pro
      01000003H   PUBLIC    CODE     ---       uart0_rec_pro
      00000098H.3 SFRSYM    DATA     BIT       TB80
      000000EDH   SFRSYM    DATA     BYTE      ADCCONT
      000000E0H.7 SFRSYM    DATA     BIT       ACC7
      00000080H   SFRSYM    DATA     BYTE      P0
      00000090H   SFRSYM    DATA     BYTE      P1
      000000A0H   SFRSYM    DATA     BYTE      P2
      00000098H.5 SFRSYM    DATA     BIT       SM20
      000000B2H   SFRSYM    DATA     BYTE      ESTCR
      000000B1H   SFRSYM    DATA     BYTE      CLKST
      000000D0H.6 SFRSYM    DATA     BIT       AC
      00000094H   SFRSYM    DATA     BYTE      PAGESEL
      000000D8H.3 SFRSYM    DATA     BIT       ERSTF
      000000E6H   SFRSYM    DATA     BYTE      PRESET0
      000000D4H   SFRSYM    DATA     BYTE      OCTRL
      000000A8H.7 SFRSYM    DATA     BIT       EA
      0000008FH   SFRSYM    DATA     BYTE      POREN
      000000C8H   SFRSYM    DATA     BYTE      PWM0CON
      000000E7H   SFRSYM    DATA     BYTE      PRESET1
      000000C9H   SFRSYM    DATA     BYTE      PWM1CON
      00000086H   SFRSYM    DATA     BYTE      BEEPCTR
      000000CAH   SFRSYM    DATA     BYTE      PWM2CON
      000000F8H.6 SFRSYM    DATA     BIT       RC32KF
LX51 LINKER/LOCATER V4.66.97.0                                                        03/02/2021  17:27:53  PAGE 28


      000000A8H   SFRSYM    DATA     BYTE      IEN0
      000000A7H   SFRSYM    DATA     BYTE      OPSET
      000000B8H   SFRSYM    DATA     BYTE      IEN1
      000000A8H.6 SFRSYM    DATA     BIT       EADC
      00000085H   SFRSYM    DATA     BYTE      DPH1
      000000B6H   SFRSYM    DATA     BYTE      ADCDR0
      000000F8H.5 SFRSYM    DATA     BIT       RC16MF
      000000B7H   SFRSYM    DATA     BYTE      ADCDR1
      00000084H   SFRSYM    DATA     BYTE      DPL1
      000000D6H   SFRSYM    DATA     BYTE      P0OD
      000000DBH   SFRSYM    DATA     BYTE      P1OD
      000000D5H   SFRSYM    DATA     BYTE      P0PD
      00000098H.4 SFRSYM    DATA     BIT       REN0
      000000ECH   SFRSYM    DATA     BYTE      P2OD
      000000DAH   SFRSYM    DATA     BYTE      P1PD
      000000E4H   SFRSYM    DATA     BYTE      P2PD
      000000D7H   SFRSYM    DATA     BYTE      P0CS
      00000097H   SFRSYM    DATA     BYTE      P0DR
      0000009EH   SFRSYM    DATA     BYTE      EUARTEN
      000000DCH   SFRSYM    DATA     BYTE      P1CS
      000000E5H   SFRSYM    DATA     BYTE      P1DR
      000000F4H   SFRSYM    DATA     BYTE      P2CS
      000000FCH   SFRSYM    DATA     BYTE      P2DR
      000000D0H.7 SFRSYM    DATA     BIT       CY
      000000D8H.0 SFRSYM    DATA     BIT       WDT0
      0000009FH   SFRSYM    DATA     BYTE      RCLTRIM
      000000D8H.1 SFRSYM    DATA     BIT       WDT1
      000000D8H.2 SFRSYM    DATA     BIT       WDT2
      00000081H   SFRSYM    DATA     BYTE      SP
      000000F1H   SFRSYM    DATA     BYTE      P0PU
      000000F2H   SFRSYM    DATA     BYTE      P1PU
      000000D1H   SFRSYM    DATA     WORD      OADR
      000000F3H   SFRSYM    DATA     BYTE      P2PU
      00000095H   SFRSYM    DATA     BYTE      D_PAGESEL
      00000093H   SFRSYM    DATA     BYTE      ADCIER
      000000D8H.6 SFRSYM    DATA     BIT       WDEN
      000000BAH   SFRSYM    DATA     BYTE      S0RELH
      00000080H.0 SFRSYM    DATA     BIT       P00
      000000D8H.7 SFRSYM    DATA     BIT       WDOF
      000000BBH   SFRSYM    DATA     BYTE      S1RELH
      00000090H.0 SFRSYM    DATA     BIT       P10
      00000080H.1 SFRSYM    DATA     BIT       P01
      00000087H   SFRSYM    DATA     BYTE      PCON
      000000C4H   SFRSYM    DATA     BYTE      PWM0DH
      000000A0H.0 SFRSYM    DATA     BIT       P20
      00000090H.1 SFRSYM    DATA     BIT       P11
      00000080H.2 SFRSYM    DATA     BIT       P02
      00000088H.0 SFRSYM    DATA     BIT       T0CLKS
      000000C6H   SFRSYM    DATA     BYTE      PWM1DH
      00000090H.2 SFRSYM    DATA     BIT       P12
      00000080H.3 SFRSYM    DATA     BIT       P03
      00000088H.4 SFRSYM    DATA     BIT       T1CLKS
      000000C7H   SFRSYM    DATA     BYTE      PWM2DH
      000000C8H.2 SFRSYM    DATA     BIT       PWM0IE
      000000AAH   SFRSYM    DATA     BYTE      S0RELL
      000000A0H.2 SFRSYM    DATA     BIT       P22
      00000090H.3 SFRSYM    DATA     BIT       P13
      00000080H.4 SFRSYM    DATA     BIT       P04
      00000089H   SFRSYM    DATA     BYTE      TMOD
      00000088H   SFRSYM    DATA     BYTE      TCON
      000000C8H.1 SFRSYM    DATA     BIT       PWM0IF
      0000009DH   SFRSYM    DATA     BYTE      S1RELL
      000000A0H.3 SFRSYM    DATA     BIT       P23
      00000090H.4 SFRSYM    DATA     BIT       P14
      000000C3H   SFRSYM    DATA     BYTE      PWM0DL
LX51 LINKER/LOCATER V4.66.97.0                                                        03/02/2021  17:27:53  PAGE 29


      00000090H.5 SFRSYM    DATA     BIT       P15
      000000A6H   SFRSYM    DATA     BYTE      OSTATUS
      000000C5H   SFRSYM    DATA     BYTE      PWM1DL
      000000A0H.5 SFRSYM    DATA     BIT       P25
      000000D8H.4 SFRSYM    DATA     BIT       PORF
      000000D8H   SFRSYM    DATA     BYTE      RSTSTAT
      000000CFH   SFRSYM    DATA     BYTE      PWM2DL
      000000A0H.6 SFRSYM    DATA     BIT       P26
      000000C8H.7 SFRSYM    DATA     BIT       PWM0EN
      000000A0H.7 SFRSYM    DATA     BIT       P27
      000000A8H.5 SFRSYM    DATA     BIT       EPWM
      000000D8H.5 SFRSYM    DATA     BIT       LVRF
      000000F8H   SFRSYM    DATA     BYTE      CLKCON
      000000CCH   SFRSYM    DATA     BYTE      PWM0PH
      000000CEH   SFRSYM    DATA     BYTE      PWM1PH
      000000C2H   SFRSYM    DATA     BYTE      PWM2PH
      000000F0H   SFRSYM    DATA     BYTE      B
      000000EEH   SFRSYM    DATA     BYTE      RCHDIV
      000000CBH   SFRSYM    DATA     BYTE      PWM0PL
      000000CDH   SFRSYM    DATA     BYTE      PWM1PL
      000000C1H   SFRSYM    DATA     BYTE      PWM2PL
      000000F7H   SFRSYM    DATA     BYTE      ADCSPW
      000000F8H.1 SFRSYM    DATA     BIT       XCLKEN
      000000E0H   SFRSYM    DATA     BYTE      ACC
      000000DDH   SFRSYM    DATA     BYTE      LVDCON
      000000A8H.4 SFRSYM    DATA     BIT       ES0
      000000A9H   SFRSYM    DATA     BYTE      IP0
      000000A8H.1 SFRSYM    DATA     BIT       ET0
      000000A8H.2 SFRSYM    DATA     BIT       ES1
      00000088H.3 SFRSYM    DATA     BIT       TF0
      000000F6H   SFRSYM    DATA     BYTE      ADCCSTAT
      000000B9H   SFRSYM    DATA     BYTE      IP1
      000000A8H.3 SFRSYM    DATA     BIT       ET1
      00000088H.7 SFRSYM    DATA     BIT       TF1
      00000098H.0 SFRSYM    DATA     BIT       RI0
      0000008CH   SFRSYM    DATA     BYTE      TH0
      000000C8H.0 SFRSYM    DATA     BIT       PWM0SS
      0000008DH   SFRSYM    DATA     BYTE      TH1
      00000098H.1 SFRSYM    DATA     BIT       TI0
      000000A8H.0 SFRSYM    DATA     BIT       EX0
      000000D0H.0 SFRSYM    DATA     BIT       P
      000000B8H.3 SFRSYM    DATA     BIT       EFCINTEN
      000000A2H   SFRSYM    DATA     BYTE      OINTEN
      0000008AH   SFRSYM    DATA     BYTE      TL0
      00000098H.7 SFRSYM    DATA     BIT       SM0
      0000008BH   SFRSYM    DATA     BYTE      TL1
      00000098H.6 SFRSYM    DATA     BIT       SM1
      000000FEH   SFRSYM    DATA     BYTE      ADCCDR0
      000000FFH   SFRSYM    DATA     BYTE      ADCCDR1
      000000D0H.3 SFRSYM    DATA     BIT       RS0
      00000088H.1 SFRSYM    DATA     BIT       TR0
      000000ACH   SFRSYM    DATA     BYTE      ADCGCR0
      000000D0H.4 SFRSYM    DATA     BIT       RS1
      00000088H.5 SFRSYM    DATA     BIT       TR1
      000000ADH   SFRSYM    DATA     BYTE      ADCGCR1
      000000B4H   SFRSYM    DATA     BYTE      ADCGCR2
      000000B5H   SFRSYM    DATA     BYTE      ADCGCR3
      000000F8H.3 SFRSYM    DATA     BIT       RC32KEN
      000000DEH   SFRSYM    DATA     BYTE      PCLK0
      000000DFH   SFRSYM    DATA     BYTE      PCLK1
      00000083H   SFRSYM    DATA     BYTE      DPH
      000000E9H   SFRSYM    DATA     BYTE      P0IEN
      000000F5H   SFRSYM    DATA     BYTE      ADCHL
      000000F8H.2 SFRSYM    DATA     BIT       RC16MEN
      000000EAH   SFRSYM    DATA     BYTE      P1IEN
LX51 LINKER/LOCATER V4.66.97.0                                                        03/02/2021  17:27:53  PAGE 30


      000000EBH   SFRSYM    DATA     BYTE      P2IEN
      000000B6H   SFRSYM    DATA     WORD      ADCDR
      000000B3H   SFRSYM    DATA     BYTE      XTHCTR
      00000082H   SFRSYM    DATA     BYTE      DPL
      00000099H   SFRSYM    DATA     BYTE      S0BUF
      0000009CH   SFRSYM    DATA     BYTE      S1BUF
      000000F9H   SFRSYM    DATA     BYTE      P0OEN
      000000D9H   SFRSYM    DATA     BYTE      SYSDIV
      00000098H   SFRSYM    DATA     BYTE      S0CON
      000000FAH   SFRSYM    DATA     BYTE      P1OEN
      000000A3H   SFRSYM    DATA     BYTE      OINTUS
      000000BEH   SFRSYM    DATA     BYTE      RCHTRIMH
      000000F8H.0 SFRSYM    DATA     BIT       SYSSEL
      0000009BH   SFRSYM    DATA     BYTE      S1CON
      000000FBH   SFRSYM    DATA     BYTE      P2OEN
      000000BDH   SFRSYM    DATA     BYTE      LDOTRIMH
      000000ABH   SFRSYM    DATA     BYTE      T2CON
      00000092H   SFRSYM    DATA     BYTE      DPS
      000000BFH   SFRSYM    DATA     BYTE      RCHTRIML
      000000D3H   SFRSYM    DATA     BYTE      ODATA
      00000091H   SFRSYM    DATA     BYTE      LDOTRIML
      000000E1H   SFRSYM    DATA     BYTE      P0IRQ
      000000B8H.1 SFRSYM    DATA     BIT       SPIINTEN
      000000E2H   SFRSYM    DATA     BYTE      P1IRQ
      000000E3H   SFRSYM    DATA     BYTE      P2IRQ
      000000D2H   SFRSYM    DATA     BYTE      OADRH
      000000F0H.0 SFRSYM    DATA     BIT       B0
      000000F0H.1 SFRSYM    DATA     BIT       B1
      000000F0H.2 SFRSYM    DATA     BIT       B2
      000000D1H   SFRSYM    DATA     BYTE      OADRL
      000000F0H.3 SFRSYM    DATA     BIT       B3
      000000F0H.4 SFRSYM    DATA     BIT       B4
      000000D0H.5 SFRSYM    DATA     BIT       F0
      000000F0H.5 SFRSYM    DATA     BIT       B5
      000000D0H.1 SFRSYM    DATA     BIT       F1
      000000AFH   SFRSYM    DATA     BYTE      REMAP
      000000F0H.6 SFRSYM    DATA     BIT       B6
      000000E0H.0 SFRSYM    DATA     BIT       ACC0
      000000A1H   SFRSYM    DATA     BYTE      OUS
      000000C8H.6 SFRSYM    DATA     BIT       PWM0S
      000000F0H.7 SFRSYM    DATA     BIT       B7
      000000E0H.1 SFRSYM    DATA     BIT       ACC1
      000000F8H.4 SFRSYM    DATA     BIT       XCLKF
      000000E0H.2 SFRSYM    DATA     BIT       ACC2
      0000008EH   SFRSYM    DATA     BYTE      PDSEL
      000000E0H.3 SFRSYM    DATA     BIT       ACC3
      000000D0H   SFRSYM    DATA     BYTE      PSW
      000000E0H.4 SFRSYM    DATA     BIT       ACC4
      00000098H.2 SFRSYM    DATA     BIT       RB80
      000000E0H.5 SFRSYM    DATA     BIT       ACC5
      000000FDH   SFRSYM    DATA     BYTE      ADCVREF
      000000E0H.6 SFRSYM    DATA     BIT       ACC6

      01000003H   BLOCK     CODE     ---       LVL=0
      01000003H   LINE      CODE     ---       #33
      01000003H   LINE      CODE     ---       #34
      01000003H   LINE      CODE     ---       #35
      0100001BH   LINE      CODE     ---       #36
      01000020H   LINE      CODE     ---       #37
      ---         BLOCKEND  ---      ---       LVL=0

      01001033H   BLOCK     CODE     ---       LVL=0
      01001033H   LINE      CODE     ---       #44
      01001033H   LINE      CODE     ---       #45
      01001033H   LINE      CODE     ---       #46
LX51 LINKER/LOCATER V4.66.97.0                                                        03/02/2021  17:27:53  PAGE 31


      01001038H   LINE      CODE     ---       #47
      ---         BLOCKEND  ---      ---       LVL=0

      01000F8BH   BLOCK     CODE     ---       LVL=0
      01000F8BH   LINE      CODE     ---       #55
      01000F8BH   LINE      CODE     ---       #56
      01000F8BH   LINE      CODE     ---       #57
      01000F8FH   LINE      CODE     ---       #58
      01000F98H   LINE      CODE     ---       #59
      ---         BLOCKEND  ---      ---       LVL=0

      01000CB0H   BLOCK     CODE     ---       LVL=0
      01000CB0H   BLOCK     CODE     NEAR LAB  LVL=1
      02000099H   SYMBOL    PDATA    BYTE      i
      0200009AH   SYMBOL    PDATA    WORD      adc_converte_data
      ---         BLOCKEND  ---      ---       LVL=1
      01000CB0H   LINE      CODE     ---       #70
      01000CB0H   LINE      CODE     ---       #71
      01000CB0H   LINE      CODE     ---       #76
      01000CBDH   LINE      CODE     ---       #77
      01000CC2H   LINE      CODE     ---       #93
      01000CD2H   LINE      CODE     ---       #94
      01000CD2H   LINE      CODE     ---       #96
      01000CDEH   LINE      CODE     ---       #97
      01000D12H   LINE      CODE     ---       #98
      01000D1DH   LINE      CODE     ---       #100
      01000D24H   LINE      CODE     ---       #103
      ---         BLOCKEND  ---      ---       LVL=0

      01000FDFH   BLOCK     CODE     ---       LVL=0
      01000FDFH   LINE      CODE     ---       #136
      01000FDFH   LINE      CODE     ---       #137
      01000FDFH   LINE      CODE     ---       #138
      01000FF2H   LINE      CODE     ---       #140
      ---         BLOCKEND  ---      ---       LVL=0

      ---         MODULE    ---      ---       MAIN
      01001020H   PUBLIC    CODE     ---       main
      00000098H.3 SFRSYM    DATA     BIT       TB80
      000000EDH   SFRSYM    DATA     BYTE      ADCCONT
      000000E0H.7 SFRSYM    DATA     BIT       ACC7
      00000080H   SFRSYM    DATA     BYTE      P0
      00000090H   SFRSYM    DATA     BYTE      P1
      000000A0H   SFRSYM    DATA     BYTE      P2
      00000098H.5 SFRSYM    DATA     BIT       SM20
      000000B2H   SFRSYM    DATA     BYTE      ESTCR
      000000B1H   SFRSYM    DATA     BYTE      CLKST
      000000D0H.6 SFRSYM    DATA     BIT       AC
      00000094H   SFRSYM    DATA     BYTE      PAGESEL
      000000D8H.3 SFRSYM    DATA     BIT       ERSTF
      000000E6H   SFRSYM    DATA     BYTE      PRESET0
      000000D4H   SFRSYM    DATA     BYTE      OCTRL
      000000A8H.7 SFRSYM    DATA     BIT       EA
      0000008FH   SFRSYM    DATA     BYTE      POREN
      000000C8H   SFRSYM    DATA     BYTE      PWM0CON
      000000E7H   SFRSYM    DATA     BYTE      PRESET1
      000000C9H   SFRSYM    DATA     BYTE      PWM1CON
      00000086H   SFRSYM    DATA     BYTE      BEEPCTR
      000000CAH   SFRSYM    DATA     BYTE      PWM2CON
      000000F8H.6 SFRSYM    DATA     BIT       RC32KF
      000000A8H   SFRSYM    DATA     BYTE      IEN0
      000000A7H   SFRSYM    DATA     BYTE      OPSET
      000000B8H   SFRSYM    DATA     BYTE      IEN1
      000000A8H.6 SFRSYM    DATA     BIT       EADC
      00000085H   SFRSYM    DATA     BYTE      DPH1
LX51 LINKER/LOCATER V4.66.97.0                                                        03/02/2021  17:27:53  PAGE 32


      000000B6H   SFRSYM    DATA     BYTE      ADCDR0
      000000F8H.5 SFRSYM    DATA     BIT       RC16MF
      000000B7H   SFRSYM    DATA     BYTE      ADCDR1
      00000084H   SFRSYM    DATA     BYTE      DPL1
      000000D6H   SFRSYM    DATA     BYTE      P0OD
      000000DBH   SFRSYM    DATA     BYTE      P1OD
      000000D5H   SFRSYM    DATA     BYTE      P0PD
      00000098H.4 SFRSYM    DATA     BIT       REN0
      000000ECH   SFRSYM    DATA     BYTE      P2OD
      000000DAH   SFRSYM    DATA     BYTE      P1PD
      000000E4H   SFRSYM    DATA     BYTE      P2PD
      000000D7H   SFRSYM    DATA     BYTE      P0CS
      00000097H   SFRSYM    DATA     BYTE      P0DR
      0000009EH   SFRSYM    DATA     BYTE      EUARTEN
      000000DCH   SFRSYM    DATA     BYTE      P1CS
      000000E5H   SFRSYM    DATA     BYTE      P1DR
      000000F4H   SFRSYM    DATA     BYTE      P2CS
      000000FCH   SFRSYM    DATA     BYTE      P2DR
      000000D0H.7 SFRSYM    DATA     BIT       CY
      000000D8H.0 SFRSYM    DATA     BIT       WDT0
      0000009FH   SFRSYM    DATA     BYTE      RCLTRIM
      000000D8H.1 SFRSYM    DATA     BIT       WDT1
      000000D8H.2 SFRSYM    DATA     BIT       WDT2
      00000081H   SFRSYM    DATA     BYTE      SP
      000000F1H   SFRSYM    DATA     BYTE      P0PU
      000000F2H   SFRSYM    DATA     BYTE      P1PU
      000000D1H   SFRSYM    DATA     WORD      OADR
      000000F3H   SFRSYM    DATA     BYTE      P2PU
      00000095H   SFRSYM    DATA     BYTE      D_PAGESEL
      00000093H   SFRSYM    DATA     BYTE      ADCIER
      000000D8H.6 SFRSYM    DATA     BIT       WDEN
      000000BAH   SFRSYM    DATA     BYTE      S0RELH
      00000080H.0 SFRSYM    DATA     BIT       P00
      000000D8H.7 SFRSYM    DATA     BIT       WDOF
      000000BBH   SFRSYM    DATA     BYTE      S1RELH
      00000090H.0 SFRSYM    DATA     BIT       P10
      00000080H.1 SFRSYM    DATA     BIT       P01
      00000087H   SFRSYM    DATA     BYTE      PCON
      000000C4H   SFRSYM    DATA     BYTE      PWM0DH
      000000A0H.0 SFRSYM    DATA     BIT       P20
      00000090H.1 SFRSYM    DATA     BIT       P11
      00000080H.2 SFRSYM    DATA     BIT       P02
      00000088H.0 SFRSYM    DATA     BIT       T0CLKS
      000000C6H   SFRSYM    DATA     BYTE      PWM1DH
      00000090H.2 SFRSYM    DATA     BIT       P12
      00000080H.3 SFRSYM    DATA     BIT       P03
      00000088H.4 SFRSYM    DATA     BIT       T1CLKS
      000000C7H   SFRSYM    DATA     BYTE      PWM2DH
      000000C8H.2 SFRSYM    DATA     BIT       PWM0IE
      000000AAH   SFRSYM    DATA     BYTE      S0RELL
      000000A0H.2 SFRSYM    DATA     BIT       P22
      00000090H.3 SFRSYM    DATA     BIT       P13
      00000080H.4 SFRSYM    DATA     BIT       P04
      00000089H   SFRSYM    DATA     BYTE      TMOD
      00000088H   SFRSYM    DATA     BYTE      TCON
      000000C8H.1 SFRSYM    DATA     BIT       PWM0IF
      0000009DH   SFRSYM    DATA     BYTE      S1RELL
      000000A0H.3 SFRSYM    DATA     BIT       P23
      00000090H.4 SFRSYM    DATA     BIT       P14
      000000C3H   SFRSYM    DATA     BYTE      PWM0DL
      00000090H.5 SFRSYM    DATA     BIT       P15
      000000A6H   SFRSYM    DATA     BYTE      OSTATUS
      000000C5H   SFRSYM    DATA     BYTE      PWM1DL
      000000A0H.5 SFRSYM    DATA     BIT       P25
      000000D8H.4 SFRSYM    DATA     BIT       PORF
LX51 LINKER/LOCATER V4.66.97.0                                                        03/02/2021  17:27:53  PAGE 33


      000000D8H   SFRSYM    DATA     BYTE      RSTSTAT
      000000CFH   SFRSYM    DATA     BYTE      PWM2DL
      000000A0H.6 SFRSYM    DATA     BIT       P26
      000000C8H.7 SFRSYM    DATA     BIT       PWM0EN
      000000A0H.7 SFRSYM    DATA     BIT       P27
      000000A8H.5 SFRSYM    DATA     BIT       EPWM
      000000D8H.5 SFRSYM    DATA     BIT       LVRF
      000000F8H   SFRSYM    DATA     BYTE      CLKCON
      000000CCH   SFRSYM    DATA     BYTE      PWM0PH
      000000CEH   SFRSYM    DATA     BYTE      PWM1PH
      000000C2H   SFRSYM    DATA     BYTE      PWM2PH
      000000F0H   SFRSYM    DATA     BYTE      B
      000000EEH   SFRSYM    DATA     BYTE      RCHDIV
      000000CBH   SFRSYM    DATA     BYTE      PWM0PL
      000000CDH   SFRSYM    DATA     BYTE      PWM1PL
      000000C1H   SFRSYM    DATA     BYTE      PWM2PL
      000000F7H   SFRSYM    DATA     BYTE      ADCSPW
      000000F8H.1 SFRSYM    DATA     BIT       XCLKEN
      000000E0H   SFRSYM    DATA     BYTE      ACC
      000000DDH   SFRSYM    DATA     BYTE      LVDCON
      000000A8H.4 SFRSYM    DATA     BIT       ES0
      000000A9H   SFRSYM    DATA     BYTE      IP0
      000000A8H.1 SFRSYM    DATA     BIT       ET0
      000000A8H.2 SFRSYM    DATA     BIT       ES1
      00000088H.3 SFRSYM    DATA     BIT       TF0
      000000F6H   SFRSYM    DATA     BYTE      ADCCSTAT
      000000B9H   SFRSYM    DATA     BYTE      IP1
      000000A8H.3 SFRSYM    DATA     BIT       ET1
      00000088H.7 SFRSYM    DATA     BIT       TF1
      00000098H.0 SFRSYM    DATA     BIT       RI0
      0000008CH   SFRSYM    DATA     BYTE      TH0
      000000C8H.0 SFRSYM    DATA     BIT       PWM0SS
      0000008DH   SFRSYM    DATA     BYTE      TH1
      00000098H.1 SFRSYM    DATA     BIT       TI0
      000000A8H.0 SFRSYM    DATA     BIT       EX0
      000000D0H.0 SFRSYM    DATA     BIT       P
      000000B8H.3 SFRSYM    DATA     BIT       EFCINTEN
      000000A2H   SFRSYM    DATA     BYTE      OINTEN
      0000008AH   SFRSYM    DATA     BYTE      TL0
      00000098H.7 SFRSYM    DATA     BIT       SM0
      0000008BH   SFRSYM    DATA     BYTE      TL1
      00000098H.6 SFRSYM    DATA     BIT       SM1
      000000FEH   SFRSYM    DATA     BYTE      ADCCDR0
      000000FFH   SFRSYM    DATA     BYTE      ADCCDR1
      000000D0H.3 SFRSYM    DATA     BIT       RS0
      00000088H.1 SFRSYM    DATA     BIT       TR0
      000000ACH   SFRSYM    DATA     BYTE      ADCGCR0
      000000D0H.4 SFRSYM    DATA     BIT       RS1
      00000088H.5 SFRSYM    DATA     BIT       TR1
      000000ADH   SFRSYM    DATA     BYTE      ADCGCR1
      000000B4H   SFRSYM    DATA     BYTE      ADCGCR2
      000000B5H   SFRSYM    DATA     BYTE      ADCGCR3
      000000F8H.3 SFRSYM    DATA     BIT       RC32KEN
      000000DEH   SFRSYM    DATA     BYTE      PCLK0
      000000DFH   SFRSYM    DATA     BYTE      PCLK1
      00000083H   SFRSYM    DATA     BYTE      DPH
      000000E9H   SFRSYM    DATA     BYTE      P0IEN
      000000F5H   SFRSYM    DATA     BYTE      ADCHL
      000000F8H.2 SFRSYM    DATA     BIT       RC16MEN
      000000EAH   SFRSYM    DATA     BYTE      P1IEN
      000000EBH   SFRSYM    DATA     BYTE      P2IEN
      000000B6H   SFRSYM    DATA     WORD      ADCDR
      000000B3H   SFRSYM    DATA     BYTE      XTHCTR
      00000082H   SFRSYM    DATA     BYTE      DPL
      00000099H   SFRSYM    DATA     BYTE      S0BUF
LX51 LINKER/LOCATER V4.66.97.0                                                        03/02/2021  17:27:53  PAGE 34


      0000009CH   SFRSYM    DATA     BYTE      S1BUF
      000000F9H   SFRSYM    DATA     BYTE      P0OEN
      000000D9H   SFRSYM    DATA     BYTE      SYSDIV
      00000098H   SFRSYM    DATA     BYTE      S0CON
      000000FAH   SFRSYM    DATA     BYTE      P1OEN
      000000A3H   SFRSYM    DATA     BYTE      OINTUS
      000000BEH   SFRSYM    DATA     BYTE      RCHTRIMH
      000000F8H.0 SFRSYM    DATA     BIT       SYSSEL
      0000009BH   SFRSYM    DATA     BYTE      S1CON
      000000FBH   SFRSYM    DATA     BYTE      P2OEN
      000000BDH   SFRSYM    DATA     BYTE      LDOTRIMH
      000000ABH   SFRSYM    DATA     BYTE      T2CON
      00000092H   SFRSYM    DATA     BYTE      DPS
      000000BFH   SFRSYM    DATA     BYTE      RCHTRIML
      000000D3H   SFRSYM    DATA     BYTE      ODATA
      00000091H   SFRSYM    DATA     BYTE      LDOTRIML
      000000E1H   SFRSYM    DATA     BYTE      P0IRQ
      000000B8H.1 SFRSYM    DATA     BIT       SPIINTEN
      000000E2H   SFRSYM    DATA     BYTE      P1IRQ
      000000E3H   SFRSYM    DATA     BYTE      P2IRQ
      000000D2H   SFRSYM    DATA     BYTE      OADRH
      000000F0H.0 SFRSYM    DATA     BIT       B0
      000000F0H.1 SFRSYM    DATA     BIT       B1
      000000F0H.2 SFRSYM    DATA     BIT       B2
      000000D1H   SFRSYM    DATA     BYTE      OADRL
      000000F0H.3 SFRSYM    DATA     BIT       B3
      000000F0H.4 SFRSYM    DATA     BIT       B4
      000000D0H.5 SFRSYM    DATA     BIT       F0
      000000F0H.5 SFRSYM    DATA     BIT       B5
      000000D0H.1 SFRSYM    DATA     BIT       F1
      000000AFH   SFRSYM    DATA     BYTE      REMAP
      000000F0H.6 SFRSYM    DATA     BIT       B6
      000000E0H.0 SFRSYM    DATA     BIT       ACC0
      000000A1H   SFRSYM    DATA     BYTE      OUS
      000000C8H.6 SFRSYM    DATA     BIT       PWM0S
      000000F0H.7 SFRSYM    DATA     BIT       B7
      000000E0H.1 SFRSYM    DATA     BIT       ACC1
      000000F8H.4 SFRSYM    DATA     BIT       XCLKF
      000000E0H.2 SFRSYM    DATA     BIT       ACC2
      0000008EH   SFRSYM    DATA     BYTE      PDSEL
      000000E0H.3 SFRSYM    DATA     BIT       ACC3
      000000D0H   SFRSYM    DATA     BYTE      PSW
      000000E0H.4 SFRSYM    DATA     BIT       ACC4
      00000098H.2 SFRSYM    DATA     BIT       RB80
      000000E0H.5 SFRSYM    DATA     BIT       ACC5
      000000FDH   SFRSYM    DATA     BYTE      ADCVREF
      000000E0H.6 SFRSYM    DATA     BIT       ACC6

      01001020H   BLOCK     CODE     ---       LVL=0
      01001020H   LINE      CODE     ---       #15
      01001020H   LINE      CODE     ---       #16
      01001020H   LINE      CODE     ---       #17
      01001023H   LINE      CODE     ---       #19
      01001026H   LINE      CODE     ---       #21
      01001029H   LINE      CODE     ---       #23
      01001029H   LINE      CODE     ---       #24
      01001029H   LINE      CODE     ---       #26
      ---         BLOCKEND  ---      ---       LVL=0

      ---         MODULE    ---      ---       ?C?FPMUL
      01000036H   PUBLIC    CODE     ---       ?C?FPMUL

      ---         MODULE    ---      ---       ?C?FPDIV
      0100013FH   PUBLIC    CODE     ---       ?C?FPDIV

LX51 LINKER/LOCATER V4.66.97.0                                                        03/02/2021  17:27:53  PAGE 35


      ---         MODULE    ---      ---       ?C?FCAST
      010001E6H   PUBLIC    CODE     ---       ?C?FCASTC
      010001E1H   PUBLIC    CODE     ---       ?C?FCASTI
      010001DCH   PUBLIC    CODE     ---       ?C?FCASTL

      ---         MODULE    ---      ---       PRINTF
      0200009CH   PUBLIC    PDATA    ---       ?_PRINTF?BYTE
      0200009CH   PUBLIC    PDATA    ---       ?_SPRINTF?BYTE
      01000818H   PUBLIC    CODE     ---       _PRINTF
      01000812H   PUBLIC    CODE     ---       _SPRINTF

      ---         MODULE    ---      ---       ?C?FPGETOPN
      0100021AH   PUBLIC    CODE     ---       ?C?FPGETOPN2
      0100024FH   PUBLIC    CODE     ---       ?C?FPNANRESULT
      01000259H   PUBLIC    CODE     ---       ?C?FPOVERFLOW
      01000231H   PUBLIC    CODE     ---       ?C?FPRESULT
      01000245H   PUBLIC    CODE     ---       ?C?FPRESULT2
      01000256H   PUBLIC    CODE     ---       ?C?FPUNDERFLOW

      ---         MODULE    ---      ---       ?C?FPROUND
      01000264H   PUBLIC    CODE     ---       ?C?FPROUND

      ---         MODULE    ---      ---       ?C?FPCONVERT
      01000293H   PUBLIC    CODE     ---       ?C?FPCONVERT

      ---         MODULE    ---      ---       ?C?FPADD
      0100039DH   PUBLIC    CODE     ---       ?C?FPADD
      01000399H   PUBLIC    CODE     ---       ?C?FPSUB

      ---         MODULE    ---      ---       ?C?FTNPWR
      010004BEH   PUBLIC    CODE     ---       ?C?FTNPWR

      ---         MODULE    ---      ---       ?C_INIT
      01000C6BH   PUBLIC    CODE     ---       ?C_START

      ---         MODULE    ---      ---       ?C?CLDPTR
      010004FEH   PUBLIC    CODE     ---       ?C?CLDPTR

      ---         MODULE    ---      ---       ?C?CLDOPTR
      01000517H   PUBLIC    CODE     ---       ?C?CLDOPTR

      ---         MODULE    ---      ---       ?C?CSTPTR
      01000544H   PUBLIC    CODE     ---       ?C?CSTPTR

      ---         MODULE    ---      ---       ?C?LADD
      01000556H   PUBLIC    CODE     ---       ?C?LADD

      ---         MODULE    ---      ---       ?C?LMUL
      01000563H   PUBLIC    CODE     ---       ?C?LMUL

      ---         MODULE    ---      ---       ?C?ULDIV
      010005EEH   PUBLIC    CODE     ---       ?C?ULDIV

      ---         MODULE    ---      ---       ?C?LNEG
      01000680H   PUBLIC    CODE     ---       ?C?LNEG

      ---         MODULE    ---      ---       ?C?ULCMP
      0100068EH   PUBLIC    CODE     ---       ?C?ULCMP

      ---         MODULE    ---      ---       ?C?ULSHR
      0100069FH   PUBLIC    CODE     ---       ?C?ULSHR

      ---         MODULE    ---      ---       ?C?LLDOPTR
      010006B2H   PUBLIC    CODE     ---       ?C?LLDOPTR

LX51 LINKER/LOCATER V4.66.97.0                                                        03/02/2021  17:27:53  PAGE 36


      ---         MODULE    ---      ---       ?C?LLDPDATA
      010006E2H   PUBLIC    CODE     ---       ?C?LLDPDATA

      ---         MODULE    ---      ---       ?C?LLDPDATA0
      010006EEH   PUBLIC    CODE     ---       ?C?LLDPDATA0

      ---         MODULE    ---      ---       ?C?LLDIPDATA
      01000704H   PUBLIC    CODE     ---       ?C?LLDIPDATA
      010006FBH   PUBLIC    CODE     ---       ?C?LLDIPDATA1
      010006FDH   PUBLIC    CODE     ---       ?C?LLDIPDATA8

      ---         MODULE    ---      ---       ?C?LSTPDATA
      0100071BH   PUBLIC    CODE     ---       ?C?LSTPDATA

      ---         MODULE    ---      ---       ?C?LSTKPDATA
      01000727H   PUBLIC    CODE     ---       ?C?LSTKPDATA

      ---         MODULE    ---      ---       ?C?PLDPDATA
      01000740H   PUBLIC    CODE     ---       ?C?PLDPDATA

      ---         MODULE    ---      ---       ?C?PLDIPDATA
      01000749H   PUBLIC    CODE     ---       ?C?PLDIPDATA

      ---         MODULE    ---      ---       ?C?PSTPDATA
      01000759H   PUBLIC    CODE     ---       ?C?PSTPDATA

      ---         MODULE    ---      ---       ?C?CCASE
      01000762H   PUBLIC    CODE     ---       ?C?CCASE

      ---         MODULE    ---      ---       ?C?ICALL
      01000788H   PUBLIC    CODE     ---       ?C?ICALL
      0100078CH   PUBLIC    CODE     ---       ?C?ICALL2

      ---         MODULE    ---      ---       ?C?DPSEL
      00000092H   PUBLIC    DATA     ---       ?C?DPSEL

      ---         MODULE    ---      ---       ?C?LLDIDATA
      0100078EH   PUBLIC    CODE     ---       ?C?LLDIDATA

      ---         MODULE    ---      ---       ?C?LLDXDATA
      0100079AH   PUBLIC    CODE     ---       ?C?LLDXDATA

      ---         MODULE    ---      ---       ?C?LLDCODE
      010007A6H   PUBLIC    CODE     ---       ?C?LLDCODE

Program Size: data=15.1 xdata=193 const=142 code=4157
LX51 RUN COMPLETE.  0 WARNING(S),  0 ERROR(S)
